:100000000C94FB0A0C94200B0C94200B0C94200BEA
:100010000C94200B0C94200B0C94200B0C94200BB4
:100020000C94200B0C94200B0C944D0C0C94200B76
:100030000C94200B0C94200B0C94200B0C94200B94
:100040000C94200B0C94200B0C94200B0C94200B84
:100050000C94200B0C94200B0C94200B0C94200B74
:100060000C94200B0C94200B0C94200B0C94200B64
:100070000C94200B0C94200B0C94200B0C94200B54
:100080000C94200B0C94200B0C94A3210C94200BAB
:100090000C94200B0C94200B0C94200B0C94200B34
:1000A0000C94200B0C94200B0C94200B0C94200B24
:1000B0000C94200B0C94200B0C94200B0C947022AD
:1000C0000C94200B0C9432260C94200B0C94200BD7
:1000D0000C94200B0C94200B0C94200B0C94200BF4
:1000E0000C94200B0C94200B0C94200B0C94200BE4
:1000F0000C94200B0C94200B0C94200B0C94200BD4
:100100000C94200B0C94200B0C94200B0C94200BC3
:100110000C94200B0C940D260C94200B0C94200BAB
:100120000C94200B0C94200B0C94200B0C94200BA3
:100130000C94200B0C94200B0C94200B0C94DB21C2
:100140000C94D8240C94200B0C94200B0C94200BB2
:100150000C94200B0C94A2250C94200B0C94200BD7
:100160000C94200B0C94200B0C94200B0C94200B63
:100170000C94200B0C94200B0C94200B0C94200B53
:100180000C94200B0C94200B0C94200B0C94200B43
:100190000C94200B0C94200B0C94200B0C94200B33
:1001A0000C94200B0C94200B0C94200B0C94200B23
:1001B0000C94200B0C94200B0C94200B0C94200B13
:1001C0000C94200B0C94200B0C94200B0C94200B03
:1001D0000C94200B0C94200B0C94200B0C94200BF3
:1001E0000C94200B0C94200B0C94200B0C94200BE3
:1001F0000C94200B0C94C3420C94200B1E03430060
:10020000680061006D0065006C0065006F006E00A5
:100210002D004D0069006E00690000002A034B00AC
:10022000610073007000650072002000260020004D
:100230004F007300770061006C00640020004700ED
:100240006D006200480000000403090409023E003A
:10025000020100C03209040000010202010005246D
:10026000001001042402060524060001070582038C
:100270000800FF09040100020A000000070504024B
:10028000100005070583021000051201100102008D
:100290000008D016B20401000102DC01F70CF80CD2
:1002A000F90CFA0CFB0CFC0CFD0CFE0C010D020D04
:1002B0000000000131239D23BC23D328D928DD2849
:1002C000FD0CDE289D2AB02A4000070031239D2323
:1002D000BC23F02A0E2B122BFD0C132BF1310D3207
:1002E0000004040031239D23BC23F02A0E2B122B83
:1002F000FD0C132BF1310D320004070031239D2337
:10030000BC23FF2A0E2B122BFD0C132BF1310D32C7
:100310000010040031239D23BC23FF2A0E2B122B37
:10032000FD0C132BF1310D320010070031239D23FA
:10033000BC23FA0CFB0CFC0CFD0CFE0C010D020D99
:10034000000000014D24C6240527353538354535D4
:1003500046356B35010D020D00000000004E4F4E7A
:100360004500000000000000000000000000000048
:1003700000000000000000000000000000014D46E9
:100380005F554C5452414C4947485400000000000E
:100390000000000000000000000000000000024D0E
:1003A000465F434C41535349435F314B00000000CB
:1003B000000000000000000000000000000000033A
:1003C0004D465F434C41535349435F314B5F374286
:1003D000000000000000000000000000000000001D
:1003E000044D465F434C41535349435F344B000037
:1003F00000000000000000000000000000000000FD
:1004000000054D465F434C41535349435F344B5FB6
:100410003742000000000000000000000000000063
:1004200000000649534F3134343433415F534E4951
:100430004646000000000000000000000000000030
:100440000000000749534F3134343433415F524583
:100450004144455200000000000000000000000080
:100460000000000001000001000101000001010086
:100470000100000100010100010000010100000174
:100480000001010000010100010000010100000164
:100490000001010001000001000101000001010054
:1004A0000100000100010100010000010100000144
:1004B0000001010001000001000101000001010034
:1004C0000100000101000001000101000001010024
:1004D0000100000100010100010000010100000114
:1004E0000001010000010100010000010100000104
:1004F00000010100010000010001010000010100F4
:1005000001000001010000010001010000010100E3
:1005100001000001000101000100000101000001D3
:1005200000010100010000010001010000010100C3
:1005300001000001000101000100000101000001B3
:1005400000010100000101000100000101000001A3
:100550000001010001000001000101000001010093
:1005600001000001008040C020A060E0109050D049
:1005700030B070F0088848C828A868E8189858D89B
:1005800038B878F8048444C424A464E4149454D49B
:1005900034B474F40C8C4CCC2CAC6CEC1C9C5CDC3B
:1005A0003CBC7CFC028242C222A262E2129252D283
:1005B00032B272F20A8A4ACA2AAA6AEA1A9A5ADA3B
:1005C0003ABA7AFA068646C626A666E6169656D63B
:1005D00036B676F60E8E4ECE2EAE6EEE1E9E5EDEDB
:1005E0003EBE7EFE018141C121A161E1119151D147
:1005F00031B171F1098949C929A969E9199959D90B
:1006000039B979F9058545C525A565E5159555D50A
:1006100035B575F50D8D4DCD2DAD6DED1D9D5DDDAA
:100620003DBD7DFD038343C323A363E3139353D3F2
:1006300033B373F30B8B4BCB2BAB6BEB1B9B5BDBAA
:100640003BBB7BFB078747C727A767E7179757D7AA
:1006500037B777F70F8F4FCF2FAF6FEF1F9F5FDF4A
:100660003FBF7FFF004E4F4E4500000000000000DE
:10067000000000000000000000000000000000007A
:100680000000000000015549445F52414E444F4D67
:10069000000000000000000000000000000000005A
:1006A000000000000000025549445F4C4546545F7D
:1006B000494E4352454D454E540000000000000095
:1006C00000000000000000035549445F52494748BC
:1006D000545F494E4352454D454E540000000000C2
:1006E0000000000000000000045549445F4C4546EE
:1006F000545F44454352454D454E540000000000B0
:10070000000000000000000000055549445F524908
:100710004748545F44454352454D454E5400000000
:1007200000000000000000000000064359434C4553
:100730005F53455454494E475300000000000000E9
:1007400000000000000000000000000753544F525A
:10075000455F4D454D000000000000000000000016
:1007600000000000000000000000000008524543A7
:10077000414C4C5F4D454D00000000000000000062
:100780000000000000000000000000000009544FBD
:1007900047474C455F4649454C4400000000000077
:1007A00000000000000000000000000000000A53EC
:1007B000544F52455F4C4F470000000000000000BE
:1007C0000000000000000000000000000000000029
:1007D0004F4646000000000000000000000000003E
:1007E0000000000000000000000000000000000009
:1007F000014D454D4F52590000000000000000001F
:1008000000000000000000000000000000000000E8
:1008100000024C49564500000000000000000000A6
:1008200000000000000000000000000000000000C8
:100830000000004E4F4E4500000000000000000088
:1008400000000000000000000000000000000000A8
:1008500000000001504F5745524544000000000081
:100860000000000000000000000000000000000088
:1008700000000000025445524D494E414C5F434F29
:100880004E4E0000000000000000000000000000CC
:100890000000000000035445524D494E414C5F5248
:1008A0005854580000000000000000000000000044
:1008B0000000000000000453455454494E475F4374
:1008C00048414E47450000000000000000000000C5
:1008D00000000000000000054D454D4F52595F5388
:1008E000544F52454400000000000000000000008A
:1008F0000000000000000000064D454D4F52595FBA
:100900004348414E474544000000000000000000FD
:1009100000000000000000000008434F4445435F12
:10092000525800000000000000000000000000001D
:100930000000000000000000000009434F44454350
:100940005F5458000000000000000000000000009C
:100950000000000000000000000000074649454C70
:10096000445F4445544543544544000000000000A2
:100970000000000000000000000000000A4C4F478B
:100980004D454D5F46554C4C0000000000000000F6
:100990000000000000000000000000000025632CA3
:1009A000256300416E7920696E7465676572206603
:1009B000726F6D203020746F2025752E2052656671
:1009C0006572656E636520766F6C7461676520770C
:1009D000696C6C2062652028564343202A205448C5
:1009E000524553484F4C44202F203430393529206C
:1009F0006D562E0025750030203D206E6F207469E5
:100A00006D656F75740D0A312D363030203D203103
:100A10003030206D73202D203630303030206D7313
:100A20002074696D656F7574002575206D730025E0
:100A3000342E345800253575206D56002575002557
:100A4000750025750025632C25630052414E444FE7
:100A50004D004E4F205549442E004368616D656C32
:100A6000656F6E4D696E692052657647202553206B
:100A70007573696E67204C55464120255320636F7E
:100A80006D70696C65642077697468204156522DD9
:100A90004743432025532E204261736564206F6EC7
:100AA00020746865206F70656E2D736F7572636555
:100AB000204E464320746F6F6C204368616D656CF7
:100AC000656F6E4D696E692E2068747470733A2F6D
:100AD0002F6769746875622E636F6D2F656D73651E
:100AE000632F4368616D656C656F6E4D696E69203B
:100AF000636F6D6D697420255300313631303234A7
:100B00000031353131313500342E392E320032305A
:100B10003035663436000D0A000D0A000D0A000D4E
:100B20000A000D0A000D0A00643130303A4F4B00C4
:100B300000000000000000000000000000000000B5
:100B4000000000000000000000653130313A4F4BDA
:100B500020574954482054455854000000000000D4
:100B6000000000000000000000006E3131303A57F4
:100B7000414954494E4720464F5220584D4F444515
:100B80004D00000000000000000000C83230303A84
:100B9000554E4B4E4F574E20434F4D4D414E440006
:100BA000000000000000000000000000C9323031E9
:100BB0003A494E56414C494420434F4D4D414E44D5
:100BC00020555341474500000000000000CA323064
:100BD000323A494E56414C494420504152414D45CC
:100BE0005445520000000000000000000000783171
:100BF00032303A46414C53450000000000000000EE
:100C0000000000000000000000000000000000796B
:100C10003132313A545255450000000000000000C6
:100C200000000000000000000000000000000000C4
:100C3000CB3230333A54494D454F555400000000F3
:100C400000000000000000000000000000000000A4
:100C50000056455253494F4E00000000000000006E
:100C6000000000000000001418434F4E46494700A2
:100C7000000000000000000000000000003C1836EA
:100C8000185549440000000000000000000000006A
:100C9000000000000092185318524541444F4E4C3A
:100CA00059000000000000000000000000F018E4FF
:100CB0001855504C4F414400000000000000000057
:100CC000001D19000000000000444F574E4C4F41DA
:100CD0004400000000000000002219000000000095
:100CE0000052455345540000000000000000000081
:100CF00000271900000000000055504752414445AC
:100D00000000000000000000003219000000000098
:100D1000004D454D53495A450000000000000000B9
:100D2000000000000000003D1955494453495A4550
:100D3000000000000000000000000000000000555E
:100D40001952425554544F4E00000000000000005C
:100D5000000000000072196B1952425554544F4E56
:100D60005F4C4F4E4700000000000000008E1987C6
:100D7000194C425554544F4E000000000000000032
:100D80000000000000AA19A3194C425554544F4EBC
:100D90005F4C4F4E470000000000000000C619BF26
:100DA000194C4544475245454E00000000000000E4
:100DB0000000000000E219DB194C45445245440094
:100DC00000000000000000000000000000FE19F715
:100DD000194C4F474D4F44450000000000000000F3
:100DE0000000000000181A131A4C4F474D454D00E3
:100DF0000000000000000000000000000000002DC6
:100E00001A4C4F47444F574E4C4F4144000000008E
:100E100000471A0000000000004C4F4753544F5247
:100E20004500000000000000004C1A000000000017
:100E3000004C4F47434C4541520000000000000069
:100E4000004F1A00000000000053455454494E471B
:100E500000000000000000000000000000571A52CF
:100E60001A434C4541520000000000000000000001
:100E700000601A00000000000053544F524500006B
:100E8000000000000000000000641A0000000000E4
:100E900000524543414C4C0000000000000000009F
:100EA00000681A0000000000004348415247494EC4
:100EB0004700000000000000000000000000006C7F
:100EC0001A48454C500000000000000000000000DF
:100ED00000741A0000000000005253534900000043
:100EE000000000000000000000000000000000B052
:100EF0001A5359535449434B0000000000000000AE
:100F000000000000000000E31A53454E445F5241C8
:100F10005700000000000000000000891B000000D6
:100F20000053454E44000000000000000000000097
:100F3000000000FF1A0000000047455455494400D6
:100F4000000000000000000000451C000000000040
:100F50000044554D505F4D46550000000000000014
:100F600000281C0000000000004944454E5449463A
:100F7000590000000000000000621C00000000009A
:100F80000054494D454F555400000000000000003A
:100F900000000000009F1C7F1C5448524553484FDE
:100FA0004C440000000000000000000000031DEBA6
:100FB0001C4649454C4400000000000000000000B1
:100FC00000000000004F1D791D000000000000001F
:100FD0000000000000000000000000000000000011
:100FE00000040001090100000000000000000000F2
:100FF00000000000000000004E58500000000000FB
:1010000000000000000000004D4946415245204DBF
:10101000696E690000000000000000000000000090
:1010200000000000000000000000000000000000C0
:1010300000000000000000000000000000000000B0
:101040000000000000000000040001080100000092
:101050000000000000000000000000000000004E42
:101060005850000000000000000000000000004D8B
:10107000494641524520436C617373696320316B6B
:101080000000000000000000000000000000000060
:101090000000000000000000000000000000000050
:1010A000000000000000000000000000000000023E
:1010B0000001180100000000000000000000000016
:1010C0000000000000004E5850000000000000002A
:1010D0000000000000004D494641524520436C612C
:1010E0007373696320346B0000000000000000008F
:1010F00000000000000000000000000000000000F0
:1011000000000000000000000000000000000000DF
:101110000000000000004400010001000000000089
:10112000000000000000000000000000004E5850C9
:10113000000000000000000000000000004D4946D3
:1011400041524520556C7472616C69676874000087
:10115000000000000000000000000000000000008F
:10116000000000000000000000000000000000007F
:101170000000000000000000000000000044030127
:10118000200175778102800000000000000000004F
:10119000000005004E585000000000000000000054
:1011A000000000004D4946415245204445534669E0
:1011B0007265000000000000000000000000000058
:1011C000000000000000000000000000000000001F
:1011D000000000000000000000000000000000000F
:1011E00000000000440301200175778102800000A7
:1011F00000000000000000000005004E58500000F4
:1012000000000000000000000000004D494641526F
:10121000452044455346697265204556310000001B
:1012200000000000000000000000000000000000BE
:1012300000000000000000000000000000000000AE
:10124000000000000000000000000004030128016D
:101250003877B14A434F503331000000000000009E
:10126000090149424D00000000000000000000009C
:1012700000004A434F5033310000000000000000DE
:10128000000000000000000000000000000000005E
:10129000000000000000000000000000000000004E
:1012A000000000000000000000000000000000003E
:1012B000000048000120017877B1024A434F507680
:1012C000323431000000000C0149424D00000000A2
:1012D0000000000000000000004A434F503331205E
:1012E00076322E342E310000000000000000000095
:1012F00000000000000000000000000000000000EE
:1013000000000000000000000000000000000000DD
:1013100000000000000000000048000120013833F8
:10132000B14A434F503431563232000000000C01B4
:1013300049424D00000000000000000000000000D5
:101340004A434F5034312076322E320000000000E4
:10135000000000000000000000000000000000008D
:10136000000000000000000000000000000000007D
:10137000000000000000000000000000000000006D
:1013800004000128013833B14A434F5034315632FA
:1013900033310000000D0149424D00000000000003
:1013A000000000000000004A434F503431207632E4
:1013B0002E332E310000000000000000000000006D
:1013C000000000000000000000000000000000001D
:1013D000000000000000000000000000000000000D
:1013E000000000000000000400018801000000006F
:1013F0000000000000000000000000000000496E36
:1014000066696E656F6E00000000000000004D49C7
:101410004641524520436C617373696320316B0010
:1014200000000000000000000000000000000000BC
:1014300000000000000000000000000000000000AC
:10144000000000000000000000000000000002009A
:1014500001980100000000000000000000000000F2
:10146000000000000047656D706C7573000000009F
:1014700000000000004D50434F53000000000000EA
:10148000000000000000000000000000000000005C
:10149000000000000000000000000000000000004C
:1014A000000000000000000000000000000000003C
:1014B0000000000000000C0100000000000000001F
:1014C000000000000000000000000000496E6E6F88
:1014D000766973696F6E2052265400004A657765FD
:1014E0006C00000000000000000000000000000090
:1014F00000000000000000000000000000000000EC
:1015000000000000000000000000000000000000DB
:101510000000000000000000000000000200013890
:1015200001000000000000000000000000000000BA
:101530000000004E6F6B69610000000000000000B9
:101540000000004D494641524520436C6173736968
:101550006320346B202D20656D756C61746564208B
:10156000283632313220436C61737369632900007D
:10157000000000000000000000000000000000006B
:101580000000000800013801000000000000000019
:10159000000000000000000000004E6F6B69610059
:1015A000000000000000000000004D494641524587
:1015B00020436C617373696320346B202D20656D4B
:1015C000756C61746564202836313331204E464392
:1015D00029000000000000000000000000000000E2
:1015E000000000000000000000006364696E6F707E
:1015F000737578585B0011241FBECFEFCDBFDFE3BA
:10160000DEBF00E00CBF18BE19BE1ABE1BBE11E241
:10161000A0E0B0E2E4E2F9E900E00BBF02C007900D
:101620000D92A438B107D9F71BBE22E3A4E8B1E2BA
:1016300001C01D92A733B207E1F73BD00C94904C48
:1016400023C13BB78BBFFB01879196913BBF0895A8
:101650003BB78BBFCB0142E20D94F00F3BB70B01C0
:1016600043E20D94F00F3BB78BBFCB0145E20D94E5
:10167000F00F3BB746E208C02091CF0127FDFCCF19
:1016800022272093CA0108954093CA0128ED31E032
:10169000209334003093CB016091C4017091C50157
:1016A0008091C60199270895FC014093CA01849155
:1016B00008950CD10E944E150E94CD15C0D21092F3
:1016C000520684E08093420682E680938601C1E060
:1016D000C0932606C093210686E080932206C0931D
:1016E000310602E00093320610922A0613E01093AE
:1016F000290689E5809380018AE58093810180E451
:1017000080934106809346069091B200907F90931B
:10171000B2009091B20092609093B20090E39093E7
:1017200041069093460680935006C0934606009368
:1017300045061093410683E18093010821E030E0E3
:1017400020932608309327082093280830932908EF
:1017500010928C088093800810922303109221032A
:10176000D8E0D093220381E18093200380911E2052
:1017700090911F2080933803909339038CE38093DA
:101780008203D093800380938303D09381036DD130
:101790000E947817BED158D6C09300021092010261
:1017A0000093020210930402C0932002D0932102FE
:1017B000EFD718D1D2E0C1E18091030481FF24C0AA
:1017C0008091010480FDFCCFD0930304B7D10E9427
:1017D000AA1742D6FFD60E94D115E091492BF0916D
:1017E0004A2B19950E9460200E941517E091582BF2
:1017F000F091592B8781813011F4C0938C29868117
:10180000813011F4C0938B290E947C17E4D6E091BB
:10181000472BF091482B1995E091412BF091422BE9
:101820001995CACF292F33272230310559F023309B
:10183000310569F021303105F9F482E190E02AE8C0
:1018400032E01EC08EE390E02CE432E019C099270C
:101850008130910541F08230910541F0892B61F48E
:10186000E8E4F2E005C0ECE1F2E002C0ECEFF1E008
:10187000849190E09F0104C080E090E020E030E09F
:10188000FA012083318308951F920F920FB60F92B1
:10189000112408B60F9218BEFFCF1F920F920FB6F9
:1018A0000F92112408B60F9218BE8F939F938EB19A
:1018B0009FB180589F4F8EB99FB99F918F910F9084
:1018C00008BE0F900FBE0F901F9018958091780062
:1018D00083FF0AC088E08093780088ED84BF81E0B0
:1018E000809380000D94FE008BEC809352008091D9
:1018F00050008860809350008091510083FFFCCF9E
:1019000082EC80935500809150008061809350005C
:101910008091510084FFFCCF88ED84BF84E08093E8
:1019200040001EB81FB881E0809343002FE730E0ED
:1019300020930A0430930B0420930C0430930D047D
:10194000809300048093020480E88093000108954E
:1019500088ED84BF81E080937900089588ED84BF8D
:101960008BE1809380000895809150008260809385
:1019700050008091510081FFFCCF82E08093CA012A
:10198000EDE1F0E0E491E0936200ECE1F0E0E4915D
:10199000E09363001092CA0180E8809365008BEBAE
:1019A0008093660080915600897F809356008091D5
:1019B000560084608093560080916000816080931F
:1019C00060000895E0E4F0E084818E7F8483E0E6A7
:1019D000F0E080818E7F8083E0E5F0E080818D7F84
:1019E0008083089587E08093A200789408950895F5
:1019F00008950895089508950895089580E090E069
:101A00000895089508950F931F93CF93DF931F9226
:101A1000CDB7DEB70DE31BE2D8011296ED91FC9134
:101A20001397898319950E949820E091582BF09183
:101A3000592B89818583B8E18B9FB00111246456AD
:101A40007D4F48E150E0C8010E94A845D801ED91C2
:101A5000FC911995D8011696ED91FC9117970F906E
:101A6000DF91CF911F910F91199448E150E06CE9FB
:101A700072E08DE39BE20E94A845E091582BF09123
:101A8000592B8581C0CF0F931F93E091582BF09174
:101A9000592B8B019C01458168E08CE593E00E9405
:101AA000B2161F910F910895FF920F931F93CF933A
:101AB000DF931F92CDB7DEB78C019E012F5F3F4FA2
:101AC000AC0168E08CE593E00E94CA16F82E8823EA
:101AD00089F0898198DFF80140E08191882319F02D
:101AE0004F5F4F31D1F7E091552BF091562BB80154
:101AF00081E119958F2D0F90DF91CF911F910F915B
:101B0000FF9008959B01AC0168E08CE593E00C9494
:101B1000F11608950C949A4508951F93CF93DF937F
:101B2000C82FD92F162F180F1C1721F00E949A4585
:101B30008993FACFDF91CF911F9108950E949A4522
:101B40000E949A450E949A450C949A45EF92FF9202
:101B50000F931F93CF93DF937C0161507109FA01BA
:101B60008A01020F131FDC0140E050E0E017F1078B
:101B7000F1F062307105D8F09191392F32953F70B4
:101B80003A3010F4305D01C0395C3C939F709A305C
:101B900010F4905D01C0995C9701240F351FE90195
:101BA00099831296625071094E5F5F4FDFCF1C928E
:101BB000CA01DF91CF911F910F91FF90EF9008958F
:101BC000CF93DF93EC01DA01E0E0F0E04C914423A5
:101BD00091F111969C911197992339F1E617F70726
:101BE00021F180ED840F8A3020F08FEB840F863056
:101BF000D0F480ED890F8A3020F02FEB290F2630AA
:101C000090F4242F30E0413410F02753310922950D
:101C1000207F913410F4982F01C09753292B2993DA
:101C200031961296D3CF80E004C011968C91811129
:101C300002C090E001C0CF01DF91CF910895E0E6AE
:101C4000F6E080E1858382E0868388E085838AE10F
:101C50008183E0EAF9E01682178280EC858388E1CF
:101C60008483E0E0F1E0128A8BE6838B148A158A84
:101C700020EA208F99E0918F128E148E158E168E89
:101C800084E0808B12A23CE633A314A215A210A616
:101C900011A612A624A795A716A680A308954115FC
:101CA000510509F449C020E12093660623E0209302
:101CB000A0092091A10927FFFCCF2091A0097093D2
:101CC000A0092091A10927FFFCCF2091A0096093D2
:101CD000A0092091A10927FFFCCF2091A00921E0B4
:101CE0002093120180931C0190931D0140931401D5
:101CF000509315011092220184E891E2809328010B
:101D00009093290140932401509325018091100163
:101D10008068809310018091200180688093200169
:101D20008091100187FDFCCF80E3809311018093A7
:101D3000210180E18093650608954115510509F45C
:101D400069C020E12093660626E02093A009209137
:101D5000A10927FFFCCF2091A00920E1209365066F
:101D6000000000002093660622E02093A009209145
:101D7000A10927FFFCCF2091A0097093A009209111
:101D8000A10927FFFCCF2091A0096093A009209111
:101D9000A10927FFFCCF2091A0091092120124E88D
:101DA00031E220931C0130931D01409314015093A4
:101DB000150120E1209322018093280190932901AD
:101DC00040932401509325018091100180688093F5
:101DD0001001809120018068809320018091100182
:101DE00087FDFCCF80E3809311018093210180E186
:101DF00080936506E091582BF091592B87818630AE
:101E000019F481E180938C298681863019F481E16F
:101E100080938B290895CF92DF92EF92FF92CF9318
:101E2000DF93C090572BD12CE12CF12C8DE0CC0C02
:101E3000DD1CEE1CFF1C8A95D1F7C114D10481E092
:101E4000E806F10408F04EC080E18093660686E063
:101E50008093A0098091A10987FFFCCF8091A00900
:101E600080E180936506000000008093660682E0B2
:101E70008093A0098091A10987FFFCCF8091A009E0
:101E80001092A0098091A10987FFFCCF8091A00941
:101E90001092A0098091A10987FFFCCF8FEFE81A6B
:101EA000F80A8091A009C0E0D0E1C701B601C9DB02
:101EB0008093A0098091A10987FFFCCF8091A009A0
:101EC0009093A0098091A10987FFFCCF8091A00980
:101ED00082E0C80ED11CE11CF11C219731F780E192
:101EE00080936506DF91CF91FF90EF90DF90CF90C8
:101EF0000895CF92DF92EF92FF92CF93DF93C0903D
:101F0000572BD12CE12CF12C8DE0CC0CDD1CEE1CE0
:101F1000FF1C8A95D1F7C114D10481E0E806F104D1
:101F200038F0DF91CF91FF90EF90DF90CF9073CF9B
:101F30008FEFE81AF80AC1E2D0E0219791F39CDB19
:101F4000C701B60185DB98DB8FEFD81AE80AF80ADB
:101F5000F4CFCF92DF92EF92FF920F931F93CF9324
:101F6000DF93C090572BD12CE12CF12C8DE0CC0CC1
:101F7000DD1CEE1CFF1C8A95D1F7C114D10481E051
:101F8000E806F10408F04FC080E18093660683E024
:101F90008093A0098091A10987FFFCCF8091A009BF
:101FA0001092A0098091A10987FFFCCF8091A00920
:101FB0001092A0098091A10987FFFCCF8FEFE81A4A
:101FC000F80A8091A009C1E2D0E0219749F154DBE1
:101FD00050DB52DB00E010E01092A0098091A109D3
:101FE00087FFFCCF6091A00970E01092A00980915A
:101FF000A10987FFFCCF8091A009782BC8012EDBB7
:102000003BDB0E5F1F4F011581E0180729F7C70161
:10201000B60129DB31DB8FEFD81AE80AF80AD5CFF1
:1020200080E180936506E091582BF091592B8781D0
:10203000863019F490E190938C299681963049F47A
:1020400020E120938B29853059F483E180938C29FA
:1020500002C08530D1F3953019F483E180938B2948
:10206000DF91CF911F910F91FF90EF90DF90CF9074
:102070000895CF92DF92EF92FF920F931F93411535
:10208000E0E25E076105710508F06BC06901E12CB3
:10209000F12C00E010E220E030E0041B150B260BD1
:1020A000370BC016D106E206F30610F4970186013D
:1020B00020E12093660626E02093A0092091A10943
:1020C00027FFFCCF2091A00920E1209365060000A6
:1020D00000002093660622E02093A0092091A10928
:1020E00027FFFCCF2091A0095093A0092091A109BE
:1020F00027FFFCCF2091A0094093A0092091A109BE
:1021000027FFFCCF2091A0091092120124E831E2B0
:1021100020931C0130931D010093140110931501AD
:1021200020E12093220180932801909329010093BC
:102130002401109325018091100180688093100183
:10214000809120018068809320018091100187FD9B
:10215000FCCF80E3809311018093210180E1809383
:10216000650681E01F910F91FF90EF90DF90CF9077
:102170000895CF92DF92EF92FF920F931F93411534
:10218000E0E25E076105710508F05DC06901E12CC0
:10219000F12C00E010E220E030E0041B150B260BD0
:1021A000370BC016D106E206F30610F4970186013C
:1021B00020E12093660623E02093A0092091A10945
:1021C00027FFFCCF2091A0095093A0092091A109DD
:1021D00027FFFCCF2091A0094093A0092091A109DD
:1021E00027FFFCCF2091A00921E0209312018093CA
:1021F0001C0190931D01009314011093150110927E
:10220000220184E891E280932801909329010093B0
:1022100024011093250180911001806880931001A2
:10222000809120018068809320018091100187FDBA
:10223000FCCF80E3809311018093210180E18093A2
:10224000650681E001C080E01F910F91FF90EF9043
:10225000DF90CF9008950F931F93CF93DF93CDB767
:10226000DEB7A097CDBFDEBF853009F4A0C0E8F48B
:10227000823009F43DC028F4813009F0DDC010E05F
:1022800028C0833009F467C0843009F0D5C0E091DC
:102290004D2BF0914E2B8E010F5F1F4FC8011995EA
:1022A0002091532BF80191E042C0883009F4B5C069
:1022B00040F4863009F4AFC0873009F0BDC049DE74
:1022C000BBC0893009F4ABC08A3009F0B5C0EED28A
:1022D000B3C08091532B181708F08CC01BDCE1E0D1
:1022E000F0E0EC0FFD1FE10FF11D80831F5FF1CFC8
:1022F000E0914D2BF0914E2B8E010F5F1F4FC801C7
:1023000019952091532BF80191E08E2F801B821795
:1023100090F4992339F0808191E08F3F09F090E0AB
:102320008F5F80833196F1CF91113AC031968E2F15
:10233000801B8217C8F3E0914F2BF091502BC801FE
:102340001995E091552BF091562B4091532BB801E4
:1023500083E1199571C0E0914D2BF0914E2BCE0188
:10236000019619958091532B41E0815008F442C0A9
:102370004423D9F3282F30E0E1E0F0E0EC0FFD1F1B
:10238000E20FF31F908141E09F3F09F040E0E1E060
:10239000F0E0EC0FFD1FE20FF31F9F5F9083E5CF8E
:1023A000808191E0811190E081508083BFCFE091E6
:1023B0004D2BF0914E2BCE01019619958091532B08
:1023C00041E08150B8F04423E1F3282F30E0E1E010
:1023D000F0E0EC0FFD1FE20FF31F908141E091113F
:1023E00040E0E1E0F0E0EC0FFD1FE20FF31F915041
:1023F0009083E7CFE0914F2BF091502BCE010196C7
:102400001995E091552BF091562B4091532BBE011D
:102410006F5F7F4F9DCF8BD30FC0FDDC0DC08091D0
:102420000008813021F480918C08833019F00E94DB
:10243000292102C00E944821A096CDBFDEBFDF91B6
:10244000CF911F910F910895E0E0F6E080E682833E
:1024500088E1868B858B0895CF93C0910806C0953F
:10246000C6FF12C0809186218A3050F08A30E1F494
:10247000E091582BF091592B8181EDDE80918621DE
:102480008F5F8093862110C08C2F807669F48091B5
:10249000862181508A3030F4E091582BF091592BED
:1024A0008081D9DE10928621C5FF12C080918521DE
:1024B0008A3050F08A30D9F4E091582BF091592BA2
:1024C0008381C9DE809185218F5F809385210FC034
:1024D000C07669F48091852181508A3030F4E09192
:1024E000582BF091592B8281B6DE10928521CF9125
:1024F00008959B01AC016BE084E696E072C420E095
:1025000030E090E0F901E80FF91FE95AF44D6383D8
:10251000265F3F4F20353105A9F708950F931F938C
:102520009B01E091582BF091592BE80FF11D8A0186
:1025300040816BE084E696E015D41F910F910895D9
:102540000F931F93CF93DF931F92CDB7DEB7082F62
:10255000AB019E012F5F3F4F6BE084E696E01AD4FB
:10256000182F882319F06981802FC9DF812F0F90E0
:10257000DF91CF911F910F9108950895EF92FF92EF
:102580000F931F93CF937B01C42F2EB13FB10091C6
:10259000080410910904022B132B682F83E090E2AA
:1025A0000E94AE436C2F83E090E20E94AE43612F05
:1025B00083E090E20E94AE43602F83E090E20E94AD
:1025C000AE436C2F70E0C701CF911F910F91FF9028
:1025D000EF9088C4089508953F924F925F926F9252
:1025E0007F928F929F92AF92BF92CF92DF92EF92A3
:1025F000FF920F931F93CF93DF937C01E90120910A
:10260000002030910120C90198532C01612C712CBC
:10261000441555056605770508F05AC04A015B0167
:102620008C0E9D1EA11CB11C84149504A604B70435
:1026300048F0841B950B8E01081B190BEC01332409
:10264000339403C000E010E0312C690180E4D81A13
:102650004601A12CB12C481559056A057B0508F5E2
:10266000CA01905C2A013B014C0E5D1E611C711C6D
:10267000481459046A047B0428F4AE01BC01C70164
:102680000EDB18C0C41AD50AA601BC01C70107DBBE
:10269000AE014C195D096BE871E2C7018C0D9D1DFF
:1026A00007C0421B530BBA0165577E4DAE01C701EF
:1026B0000E94D645311002C081E00BC001501109C3
:1026C000D8F3F801EC0FFD1FEE0DFF1D1082F6CFC1
:1026D00080E0DF91CF911F910F91FF90EF90DF90FD
:1026E000CF90BF90AF909F908F907F906F905F90B2
:1026F0004F903F900895EBE8F1E2119289E2EB38B8
:10270000F807D9F78BE891E28093892190938A2189
:1027100080E098E0809387219093882180E090E486
:102720008093002090930120E091582BF091592B39
:1027300087818A3019F480E180938C2986818A30E0
:1027400019F480E180938B290895809187219091DD
:102750008821089520E030E0F901E95AF44D87839B
:10276000265F3F4F20353105B9F7813039F018F039
:10277000823039F008958DEB92E105C08FEC93E142
:1027800002C08EEB92E18093552B9093562B0895C7
:10279000B2DFE091582BF091592B8481DBCF0F935E
:1027A0001F93CF93DF93AEB1BFB1C0910804D09116
:1027B00009042091872130918821E42FF0E08F01D6
:1027C0000C5F1F4F2017310758F1CA2BDB2B245009
:1027D00031092E1B3F0B2093872130938821A09134
:1027E0008921B0918A218C9311964C93119712965E
:1027F000DC931297CD0104968093892190938A21CE
:102800001396CC93DB01EC01415018F02D912993E4
:10281000FBCFE80FF91FE0938921F0938A2112C0C2
:1028200080E098DFE091582BF091592B87818A3016
:1028300019F481E180938C2986818A3019F481E131
:1028400080938B29DF91CF911F910F9108951F9352
:10285000CF93DF931F92CDB7DEB79E012F5F3F4F1F
:10286000AC0163E08FEC97E095D2182F882311F02C
:10287000898170DF812F0F90DF91CF911F91089593
:102880000F931F93E091582BF091592B8B019C01D2
:10289000448163E08FEC97E065D21F910F9108951A
:1028A0009B01AC0163E08FEC97E09BC2CF93DF9379
:1028B0008091872190918821811528E0920710F559
:1028C000609100207091012040E058E0481B590BB6
:1028D00080E090E8861B970B8417950798F08BE8AB
:1028E00091E22BDAC0910020D0910120D85F809135
:1028F000872190918821C81BD90BFDDEC093002051
:10290000D0930120DF91CF9108958091CF0187FD71
:10291000FCCF0895FADF8091CF0181FF0BC086E3E1
:102920008093CA01EBECF1E021E030E088ED90E02B
:1029300084BF20830895EF92FF920F931F93CF934C
:10294000DF931F921F92CDB7DEB77C018A011092F0
:10295000C20169837A83D9DF6981A62F7A81B72F73
:10296000C701800F911F26E048ED50E061E070E064
:10297000EBECF1E0E816F90689F0E092C0013F2D9A
:102980003F713093C1012093CA0144BF60833091ED
:10299000C4013D933FEFE31AF30AECCFC8010F9057
:1029A0000F90DF91CF911F910F91FF90EF900895BD
:1029B0002F923F924F925F926F927F928F929F924F
:1029C000AF92BF92CF92DF92EF92FF920F931F933D
:1029D000CF93DF9300D0CDB7DEB76A01282F2F71D8
:1029E0001C01221A310829836A837B8393DF8DDFE0
:1029F00083E38093CA011092C1011092C2016A81DF
:102A0000E62E7B81F72E860185E3582E98ED892EE0
:102A1000912C66246394712C3BECA32EBB24B394BD
:102A200043E3442E29810115110509F12093C001CA
:102A3000F70181917F018093C4010150110919F0C0
:102A40002F5F203281F72092C001832D8F718093F8
:102A5000C1015092CA01C401F50184BF608290E2B5
:102A6000290E311C52DF4092CA0120E0DCCFC601A2
:102A70002396CDBFDEBFDF91CF911F910F91FF90C5
:102A8000EF90DF90CF90BF90AF909F908F907F900E
:102A90006F905F904F903F902F90089543E550E0E6
:102AA00067E57BE280E090E046CF43E550E067E5F4
:102AB0007BE280E090E07CCFCF93DF93CFEFC80F35
:102AC000C83078F5D82F0E94982043DAC093572B4E
:102AD0008AE0C89F90011124C901865A944D8093C1
:102AE000582B9093592BF901E95AF44D80850E9497
:102AF000030DE091582BF091592B84812BDE8BD95B
:102B00008FE18D0FE091582BF091592B97819430E4
:102B100011F480938C299681943029F480938B2929
:102B200002C080E001C081E0DF91CF9108958091E3
:102B3000572B99E04AE0915099F0282F30E02F5F11
:102B40003F4F27703327822F429FF001439FF00DA4
:102B50001124E95AF44D2085222369F38F5FACCF0D
:102B60000895FC019091572B9F5C908311820895EA
:102B7000CF93FC01C081818181110CC0BF01E09124
:102B8000552BF091562B41E082E1199580ED8C0F89
:102B9000CF9192CF80E0CF91089588E18093010694
:102BA000089580918B29823191F030F48031B9F011
:102BB00050F48823A9F132C0833169F090EE980F68
:102BC000983088F02BC088E08093050627C088E005
:102BD0008093070623C08091040683FF12C088E01B
:102BE000809306061BC090918D299F5F923019F04B
:102BF00090938D2915C010928D299091040693FD14
:102C000004C088E0809305060BC098E09093060608
:102C1000803221F0815080938B2902C010928B2941
:102C200080918C29823191F030F48031C1F050F4E0
:102C30008823A9F132C0833169F090EE980F983063
:102C400088F02BC080E18093050627C080E1809347
:102C5000070623C08091040684FF12C080E18093A0
:102C600006061BC090918E299F5F923019F09093B9
:102C70008E29089510928E299091040694FD04C027
:102C800080E180930506089590E1909306068032D6
:102C900021F0815080938C29089510928C290895F9
:102CA0009B01AC016BE082E398E09BC020E030E048
:102CB000982F90718870992321F0F901E95AF44D09
:102CC0006287882321F0F901E95AF44D6187265F74
:102CD0003F4F2035310579F7992329F090E1909302
:102CE000060610928C29882329F088E08093060636
:102CF00010928B2908950F931F939B018A018031B5
:102D000031F4E091582BF091592B478107C088305E
:102D100049F4E091582BF091592B46816BE082E306
:102D200098E020D01F910F9108950F931F93CF9398
:102D3000DF931F92CDB7DEB7082FAB019E012F5F47
:102D40003F4F6BE082E398E025D0182F882319F0DD
:102D50006981802FABDF812F0F90DF91CF911F9181
:102D60000F9108950F931F93FC01662379F09491BE
:102D70006150941309C0BF016F5F7F4FA801C90163
:102D80000E94BA4581E003C0B196EFCF80E01F9169
:102D90000F910895CF92DF92EF92FF921F93CF93FE
:102DA000DF93EC017A016901162F112389F0BE012E
:102DB0006F5F7F4FC7010E94B1451150892B31F4DD
:102DC000FE01C491F601C08381E003C0A196EDCF5E
:102DD00080E0DF91CF911F91FF90EF90DF90CF9037
:102DE0000895CF930196CCE26623C9F0FC01DA0185
:102DF000AD017491772341F021153105A1F07D9348
:102E0000319621503109F4CF623030F0211531056F
:102E100051F04F5F5F4FCC9361508196E5CF232BEC
:102E200011F0FA011082CF910895809120028068FC
:102E3000809320028091230280FFFCCF81E0809369
:102E40002302A0911002B0911102AE5BB109B7FF4D
:102E500002C0A0E0B0E020E038EB4BE050E00E9480
:102E60003445E091582BF091592B61157105844F31
:102E70009140A8F48781873019F480E180938C29F0
:102E80008681873019F480E180938B298091532BC0
:102E9000882389F0E091452BF091462B1994878186
:102EA000873019F481E180938C298681873019F469
:102EB00081E180938B290895BC0183E090E20C941A
:102EC0006043CF93DF93FC016491EC01219666236C
:102ED00031F083E090E20E94AE43CE01F4CFDF9167
:102EE000CF910895AB01BC0183E090E20C948A433A
:102EF00080E2809362060895CF93DF9380918F29BB
:102F0000823029F583E090E20E9413440E94E23E61
:102F100083E090E20E942F44EC0197FD18C0E091FD
:102F2000582BF091592B8781833019F483E18093DA
:102F30008C298681833019F483E180938B298C2F2F
:102F400019D6811104C08C2FDF91CF91B7C7DF91C3
:102F5000CF91089580918F29813079F028F08230C7
:102F6000D9F0833011F12EC08091680685FF2AC008
:102F70008FE08093022081E00CC08091022081507C
:102F80008093022081111EC00E94B40C0E948D42C9
:102F900082E080938F2916C08091680685FD12C05B
:102FA0008FE08093022083E0F4CF80910220815053
:102FB00080930220811106C00E9452420E94E20CBE
:102FC00010928F2980918F29823019F423D70C9485
:102FD00060200895E091582BF091592B8781823021
:102FE00019F481E180938C298681823019F481E182
:102FF00080938B290895E091582BF091592B87816C
:10300000823019F480E180938C298681823019F412
:1030100080E180938B29089583E090E20C943B43F8
:1030200083E090E20C9482442EE03BE03F932F93A8
:1030300028E03BE03F932F9321E03BE03F932F9329
:103040002AEF3AE03F932F932AE53AE03F932F93FC
:1030500022E02F931F929F938F930E943F468DB73C
:103060009EB70E968DBF9EBF85E6089560E072E024
:103070000E94430D85E60895FB0120812F3349F41A
:103080002181211106C060E072E00E94820D85E678
:103090000895CB010E94540D882319F006DD84E6C3
:1030A00008958AEC0895EF92FF920F931F93CF93A8
:1030B000DF93CDB7DEB7A097CDBFDEBF7C01009117
:1030C000532B10E00115110591F482E59AE09F93CE
:1030D0008F9382E08F931F92FF92EF920E943F4660
:1030E0000F900F900F900F900F900F9010C0E091E5
:1030F0004D2BF0914E2BCE01019619959801AE0102
:103100004F5F5F4F60E072E0C7010E94A60D85E649
:10311000A096CDBFDEBFDF91CF911F910F91FF90A1
:10312000EF900895DF92EF92FF920F931F93CF934A
:10313000DF93CDB7DEB7A097CDBFDEBF7B01009197
:10314000532B10E06BE47AE0C7010E94B145892B54
:1031500029F5D12CED2CF12CE016F10658F40E9443
:103160008A0DE1E0F0E0EC0FFD1FEE0DFF1D808306
:10317000D394F0CFE0914F2BF091502BCE010196DC
:103180001995E091552BF091562B4091532BBE0190
:103190006F5F7F4F83E1199584E60BC0A70160E262
:1031A00070E0CE0101960E94E00D8017910711F3A7
:1031B0008AECA096CDBFDEBFDF91CF911F910F911A
:1031C000FF90EF90DF900895FC018091542B8823AD
:1031D00011F081E301C080E38083118285E60895C8
:1031E000FB012181211127C02081213321F481E0BD
:1031F0008093542B04C0203321F41092542B84E686
:1032000008952F33C1F41F9220E32F931F9221E3DF
:103210002F9325E43AE03F932F9322E02F931F92C0
:103220009F938F930E943F468DB79EB70A968DBF9E
:103230009EBF85E608958AEC089589E390E169D4FC
:103240008EE6089589EB90E17FD48EE60895E0EC58
:10325000F4E081818E7F81830E9452420E94A80CFB
:1032600084E60895E0ECF4E081818E7F81830E9402
:1032700052420E94AE0C84E60895EDE3FBE22589FC
:103280002F9324892F9322E43AE03F932F9322E057
:103290002F931F929F938F930E943F468DB79EB7A7
:1032A00008968DBF9EBF85E608952091532B1F92EF
:1032B0002F932FE33AE03F932F9322E02F931F9217
:1032C0009F938F930E943F468DB79EB708968DBF00
:1032D0009EBF85E6089540E052E0BC0180E01ED923
:1032E00085E60895FB0120812F3341F421812111CE
:1032F00005C060E072E0FDD885E6089580E020D941
:10330000882319F0D2DB84E608958AEC089540E022
:1033100052E0BC0181E002D985E60895FB012081DD
:103320002F3341F42181211105C060E072E0E1D822
:1033300085E6089581E004D9882319F0B6DB84E698
:1033400008958AEC089540E052E0BC0182E0E6D89E
:1033500085E60895FB0120812F3341F4218121115D
:1033600005C060E072E0C5D885E6089582E0E8D83F
:10337000882319F09ADB84E608958AEC089540E0EA
:1033800052E0BC0183E0CAD885E60895FB012081A4
:103390002F3341F42181211105C060E072E0A9D8EA
:1033A00085E6089583E0CCD8882319F07EDB84E697
:1033B00008958AEC089540E052E0BC0180E19BDC76
:1033C00085E60895FB0120812F3341F421812111ED
:1033D00005C060E072E064DC85E6089580E1A5DC6C
:1033E000882319F062DB84E608958AEC089540E0B2
:1033F00052E0BC0188E07FDC85E60895FB01208176
:103400002F3341F42181211105C060E072E048DCD6
:1034100085E6089588E089DC882319F046DB84E698
:1034200008958AEC089560E072E02ADA85E608954E
:10343000FB0120812F3341F42181211105C060E07F
:1034400072E02EDA85E60895CB0101DA882319F0BF
:103450002CDB84E608958AEC0895CF93DF93EC018A
:1034600074D99F938F932CE33AE03F932F9382E09C
:103470008F931F92DF93CF930E943F468DB79EB7E5
:1034800008968DBF9EBF85E6DF91CF9108958CEEA3
:1034900092E15AD38EE6089509DA84E608952BD98D
:1034A00084E6089560E072E05CDB85E60895CB0178
:1034B0005FDB882319F0F9DA84E608958AEC089531
:1034C0000E94790F84E608950E94A90F84E608956A
:1034D0000E940B0F84E608958091680680FD02C06B
:1034E00089E7089588E70895DF92EF92FF920F939E
:1034F0001F93CF93DF93EC010FEF11E081E5E82EEE
:103500008CE0F82E9CE2D92EB7018EE691E20E9463
:10351000B145892BD1F001151105B9F0DE01F70194
:103520002491ED012196C8010197222341F0013039
:10353000110529F02C93DE0131968C01F1CFDC923C
:103540008C0188E1E80EF11CDFCF2197188285E617
:10355000DF91CF911F910F91FF90EF90DF90089531
:10356000FC012091200220682093200280912302F8
:1035700080FFFCCF81E080932302A0911002B091E4
:103580001102AE5BB109B7FF02C0A0E0B0E020E0DD
:1035900038EB4BE050E00E943445AA27BB279F93AD
:1035A0008F9325E33AE03F932F9382E08F931F920E
:1035B000FF93EF930E943F468DB79EB708968DBF4D
:1035C0009EBF85E608952EB13FB140910804509109
:1035D0000904242B352B3F932F932FE23AE03F939E
:1035E0002F9322E02F931F929F938F930E943F4629
:1035F0008DB79EB708968DBF9EBF85E608950F9341
:103600001F93CF93DF931F921F92CDB7DEB78B012D
:10361000E091582BF091592B8581873009F06FC0CC
:10362000E091452BF091462B199581E08093D929A3
:1036300060E270E0C8010E94F7450097F9F4F801D4
:1036400001900020E9F73197E01BF10BE0FD59C034
:10365000F695E795E130F10539F487E090E0809345
:103660003B2B90933C2B37C053E0EE0FFF1F5A9536
:10367000E1F7E0933B2BF0933C2B2DC098012C5F9E
:103680003F4F82179307E9F5A80162E070E0CE0191
:1036900001960E94E00D898190E0982F88272A8169
:1036A000820F911D80933B2B90933C2B0B5F1F4F00
:1036B000F80101900020E9F73197E01BF10BE0FDE4
:1036C00020C0F695E79533E0EE0FFF1F3A95E1F73E
:1036D000E817F907B0F060913B2B70913C2B695FC4
:1036E0007F4F83E0769567958A95E1F7A8018BE394
:1036F0009AE20E94E00D0E947F288FEF03C089ECC0
:1037000001C08AEC0F900F90DF91CF911F910F9124
:103710000895EF92FF920F931F93CF93DF931F9221
:103720001F92CDB7DEB78B01E091582BF091592B4A
:103730008581873009F080C0E091452BF091462BC0
:10374000199582E08093D92960E270E0C8010E9457
:10375000F7457C01892B31F5F80101900020E9F74C
:103760003197E01BF10BE0FD69C0F695E795E1307C
:10377000F10539F487E090E080933B2B90933C2B4C
:1037800047C063E0EE0FFF1F6A95E1F7CF0169E0E4
:1037900070E00E942045E81BF90BE0933B2BF0936F
:1037A0003C2B36C0C8010496E816F90609F046C05D
:1037B000A80162E070E0CE0101960E94E00D29812F
:1037C00030E0322F22278A81280F311D20933B2B96
:1037D00030933C2B2730310529F0C9018770992798
:1037E000892B61F587010F5F1F4FF80101900020C1
:1037F000E9F73197E01BF10BE0FD20C0F695E79566
:1038000043E0EE0FFF1F4A95E1F7E217F307B0F030
:1038100060913B2B70913C2B695F7F4F83E07695E5
:1038200067958A95E1F7A8018BE39AE20E94E00D83
:103830000E947F288FEF03C089EC01C08AEC0F90B3
:103840000F90DF91CF911F910F91FF90EF9008950E
:10385000E091582BF091592B85818730A1F4E091AC
:10386000452BF091462B199584E08093D9290E942D
:1038700035350E947F288FE395E380939F299093AD
:10388000A0298FEF089589EC0895E091582BF091CD
:10389000592B85818730A1F4E091452BF091462B7F
:1038A000199583E08093D9290E9435350E947F289D
:1038B0008FE395E380939F299093A0298FEF08953C
:1038C00089EC0895E091582BF091592B8581873030
:1038D000A1F4E091452BF091462B199585E080935A
:1038E000D9290E9435350E947F288FE395E3809384
:1038F0009F299093A0298FEF089589EC0895E09176
:10390000582BF091592B4085518564E6649F9001B6
:10391000659F300D11243F932F9329E23AE03F93A6
:103920002F9322E02F931F929F938F930E943F46E5
:103930008DB79EB708968DBF9EBF85E60895CF933D
:10394000DF931F921F92CDB7DEB7FB0120812F338B
:10395000B1F42181211113C027EF39E03F932F9358
:1039600022E02F931F929F938F930E943F460F90C8
:103970000F900F900F900F900F9085E627C089E56C
:1039800092E089839A83CE0101969F938F938EEB69
:1039900090E29F938F937F936F930E9475460F9051
:1039A0000F900F900F900F900F90892B71F08981DD
:1039B0009A818935F2E09F0740F4E091582BF0910D
:1039C000592B8087918784E601C08AEC0F900F9075
:1039D000DF91CF91089520911F202F9320911E20D9
:1039E0002F9324EF39E03F932F9322E02F931F92E0
:1039F0009F938F930E943F468DB79EB708968DBFC9
:103A00009EBF85E60895CF93DF931F921F92CDB797
:103A1000DEB7FB0120812F33B1F42181211113C0C6
:103A20002FE02F932FEF2F9323EA39E03F932F932B
:103A300022E02F931F929F938F930E943F46CDBF0A
:103A4000DEBF85E627C019821A82CE0101969F93B8
:103A50008F938EEB90E29F938F937F936F930E944F
:103A600075460F900F900F900F900F900F90892B2D
:103A700081F089819A818115E0E19E0750F480935D
:103A800038039093390380931E2090931F2084E67F
:103A900001C08AEC0F900F90DF91CF910895FB0148
:103AA00020812F33D9F42181211121C01F9220E3DD
:103AB0002F931F9221E32F932DE939E03F932F930A
:103AC00022E02F931F929F938F930E943F468DB7C2
:103AD0009EB70A968DBF9EBF85E60895213311F4E7
:103AE000B8D303C0203319F4D3D384E608958AEC05
:103AF0000895FC0180910008813021F480918C08A8
:103B0000833011F080E301C081E38083118285E678
:103B1000089521E020939E2920939D292CE3209352
:103B20009A2925E030E02093982930939929109222
:103B3000922910929329109294291092952980939A
:103B4000902990939129089527E020939E292CE2B3
:103B500031E020939829309399291092922910925C
:103B600093291092942910929529809390299093EB
:103B700091290895CF9390919E299530E1F130F4E9
:103B8000933029F140F5913068F440C1973009F441
:103B9000A7C008F445C0983009F4AAC0993009F4C8
:103BA00032C134C1813041F4109296291092972984
:103BB00010929B2983E0FBC0843011F466E08BC037
:103BC000883109F420C18B3109F0F3C01CC1809306
:103BD0009C2984E0ECC090E040919C292FEF30E0DC
:103BE000241B31098217930721F485E0E0C0981760
:103BF00039F165E169C02091962930919729A90191
:103C00004F5F5F4F4093962950939729F901E655EE
:103C1000F44D80834038510509F0CBC086E0C7C021
:103C200020919C2990919D29291346C0EAEAFBE244
:103C300090E02CE2EA32F207D1F22191920FF9CF13
:103C400040919229509193296091942970919529DE
:103C5000E0919029F091912920E830E08AEA9BE2F6
:103C60001995C82F882311F180919D298F5F80932A
:103C70009D298091922990919329A0919429B091A6
:103C8000952980589F4FAF4FBF4F809392299093B3
:103C90009329A0939429B093952966E083E090E25C
:103CA0000E94AE4382E080939E29B1C068E183E028
:103CB00090E20E94AE430EC030E0892F90E0019761
:103CC0002817390739F466E083E090E20E94AE439A
:103CD00082E06DC068E183E090E20E94AE4393C051
:103CE000853119F410929D2909C08B3109F48BC0DC
:103CF000883109F463CF863009F05DC080919D2939
:103D00008F5F80939D2940919229509193296091D2
:103D1000942970919529E0919029F091912920E8BA
:103D200030E08AEA9BE21995C82F8823D1F161E03F
:103D300083E090E20E94AE4360919D2983E090E28F
:103D40000E94AE4360919D29609583E090E20E94BD
:103D5000AE4360E870E08AEA9BE2C4D8EAEAFBE29C
:103D600060E08CE2EA32F80719F08191680FF9CF30
:103D700083E090E20E94AE43809192299091932932
:103D8000A0919429B091952980589F4FAF4FBF4F74
:103D90008093922990939329A0939429B093952985
:103DA00036C064E083E090E20E94AE4389E08093F5
:103DB0009E29C1E02CC08531E1F761E083E090E20B
:103DC0000E94AE4360919D2983E090E20E94AE4341
:103DD00060919D29609583E090E20E94AE4360E887
:103DE00070E08AEA9BE27ED8EAEAFBE260E02CE23D
:103DF000EA32F20719F08191680FF9CF83E090E27F
:103E00000E94AE43D6CF10929E29D3CFC0E08C2F14
:103E1000CF91089580919E29813019F0873029F142
:103E2000089580919829909199299C0121503109F8
:103E30002093982930939929892B31F580919A29DB
:103E40009FEF980F90939A29882331F065E183E0E2
:103E500090E20E94AE4302C010929E2985E090E05D
:103E60008093982990939929089580919829909109
:103E700099299C012150310920939829309399293F
:103E8000892B11F410929E290895E8E2FBE020E0CE
:103E900030E09491981309C041E2429FC001439FD2
:103EA000900D1124875D944F08952F5F3F4FB19679
:103EB0002930310571F780E090E00895CF92DF92CC
:103EC000EF92FF920F931F93CF93982F9F7D915462
:103ED0009A3160F090ED980F9A3040F08F3531F0C4
:103EE000982F9D7F9D3311F08032D1F49FE9980F78
:103EF0009A3108F480522091A4293091A5292F3FAE
:103F000091E0390708F0D3C0A9014F5F5F4F40939C
:103F1000A4295093A529F901E655F44D8083C7C023
:103F20008D3009F095C0E091A429F091A529E655BE
:103F3000F44D10821092A4291092A5298091A329F2
:103F40008111B5C08091AA2B982F9F7D09F495C04F
:103F50008D7F8D3309F491C0EAEAFBE27F01C191C4
:103F6000CC2331F0CF3321F0CD3311F0C032B1F793
:103F7000F701108281E5C82E8CE0D82E00E010E019
:103F8000B6018AEA9BE20E94B145892B09F056C02E
:103F90001092AA2BCF3349F488E1809FF001819FD2
:103FA000F00D1124E959F34F18C0B7016F5F7F4F2F
:103FB000CD3349F488E1809FF001819FF00D1124F9
:103FC000EB59F34F20C0C11113C088E1809FF0016D
:103FD000819FF00D1124EF59F34F25913491211554
:103FE000310509F44DC08AEA9BE2F901199514C024
:103FF000C03209F045C088E1809FF001819FF00D3B
:104000001124ED59F34F2591349121153105C1F15A
:104010008AEA9BE2F90119958F3F99F581E0809337
:10402000A3298EB19FB12091080430910904822BFD
:10403000932B8093A1299093A22939C00F5F1F4F22
:10404000F8E1CF0ED11C0632110509F099CF15C049
:10405000883061F48091A4299091A529009739F1C5
:1040600001978093A4299093A52921C08B31F9F45D
:104070001092A4291092A5291AC088ECC0E002C0B1
:1040800089ECC1E002DF0E94611785E29BE00E949B
:104090006117CC2361F08091AA2B882341F08AEA32
:1040A0009BE20E945C1782E29BE00E94611781E024
:1040B000CF911F910F91FF90EF90DF90CF900895D7
:1040C0008091A329882399F1E091582BF091592BE5
:1040D000208531852115310551F18EB19FB1409177
:1040E000080450910904842B952B4091A1295091EB
:1040F000A229841B950B64E670E00E94204562179C
:104100007307A8F01092A3298BECBFDE0E94611701
:104110008FE19BE00E946117E0919F29F091A02917
:10412000309729F0199510929F291092A02908958F
:104130008091A3298823A9F01092A3298BECA5DEF6
:104140000E9461178FE19BE00E946117E0919F2917
:10415000F091A029309729F0199510929F2910927B
:10416000A0290895CF93DF939091A3299923A9F0D3
:10417000EB011092A32989DE0E9461178CE19BE07C
:104180000E946117209749F0CE010E945C1789E1D7
:104190009BE0DF91CF910C946117DF91CF9108954F
:1041A000EF92FF920F931F93CF937C019B0161309D
:1041B00081E0780710F020E031E08B01021B130B47
:1041C000A70160E072E08AEA9BE20E94A60D8AEAFB
:1041D0009BE20E945C17C1E0013081E01807C0F04B
:1041E0001A954C2F50E0542F4427550F569547955C
:1041F0004E0D5F1D20E032E060E072E08AEA9BE253
:104200000E94A60D8AEA9BE20E945C17CF5FE4CF72
:1042100001151105A9F0EC2FF0E0FE2FEE27FF0F9E
:10422000F695E795A7014E0F5F1F980160E072E0D9
:104230008AEA9BE20E94A60D8AEA9BE20E945C1732
:1042400086E19BE0CF911F910F91FF90EF900C942E
:10425000611780910008813021F480918C088330AF
:10426000B1F081E08093000893E090938C088093F4
:10427000A6291092A7298EB19FB1209108043091F0
:104280000904822B932B8093A8299093A929089540
:1042900010928C0810920008E6EAF9E2108211826E
:1042A00008959091A6299923F1F08091A729811171
:1042B00015C02091A6292223B9F02EB13FB140911B
:1042C000080450910904242B352B4091A8295091C2
:1042D000A929241B350B2634310530F081E0809369
:1042E000A729892F089581E00895A0E2B6E081E032
:1042F00015968C9315972AEA3DE228B939B92AE236
:104300003EE22AB93BB910B813B812B816B817B8BC
:1043100011B8E0E0F9E010A211A22FEF30E026A3DF
:1043200037A32FEF3FEF20A731A7808388E883834F
:1043300080E1848783E087831C968C931C9782E0BE
:104340001A968C9308951F920F920FB60F92112414
:1043500008B60F9218BE0BB60F921BBE8F939F9399
:10436000EF93FF93E0E0F9E013828FE790E086ABF4
:1043700097AB81E190E080AF91AFE0E0FAE010A26E
:1043800011A28FEF9FEF86A397A389E883831682FC
:1043900081E084878EE0808310922A06FF91EF915E
:1043A0009F918F910F900BBE0F9008BE0F900FBE84
:1043B0000F901F9018951F920F920FB60F92112415
:1043C00008B60F9218BE0BB60F921BBE2F933F93E9
:1043D0008F939F93EF93FF932091280693B12670BC
:1043E00081E009F080E0990F892B83B982B188239D
:1043F00009F464C012B883B18770873059F5109200
:10440000000980E180930C091092030A1B9B03C0F2
:104410008CEA94E002C08CE694E08093260A9093A4
:10442000270A82E081B981E080930C0A83E08093BF
:10443000060A86B197B1877049F090B18F5F8930D5
:1044400011F09695FBCFE8B1F9B1908381E08093AC
:10445000AA2937C093B1892F8C7099F192FB9927C3
:1044600090F981E0982781B181111BC080B18695B8
:10447000911190E8892B80B926B137B12F5F3F4F5A
:1044800026B937B927703327232BD9F4E8B1F9B10E
:104490009F012F5F3F4F28B939B9808381E081B9EF
:1044A00010C081B1813069F4EAB1FBB19F012F5F87
:1044B0003F4F2AB93BB9908311B803C082B18095B0
:1044C00082B9FF91EF919F918F913F912F910F9022
:1044D0000BBE0F9008BE0F900FBE0F901F90189547
:1044E0001F920F920FB60F92112408B60F9218BEAA
:1044F0000BB60F921BBE2F933F938F939F93EF9317
:10450000FF9381B1823008F49DC081B18D3008F0F5
:1045100099C0E1B1F0E0EE0FFF1FEC5DFF4D01909F
:10452000F081E02D19948FE790E08093260A909314
:10453000270A88C08E9A8EE0809340088FE390E02F
:104540008093260A9093270A85E06FC08E9886E0B4
:1045500081B98FEF82B914B815B8E8B1F9B180818B
:1045600080B970C0009B05C08E9A82B1809582B9D7
:1045700001C08E9887E059C0009B02C08E9801C090
:104580008E9A80B1869580B984B195B1019684B92F
:1045900095B984B195B187709927892B11F488E07A
:1045A00044C024B135B186B197B128173907B1F5A8
:1045B0002BC0EAB1FBB1309711F0808101C082B10C
:1045C000882311F08E9A01C08E9889E02EC0EAB13E
:1045D000FBB1309751F08081882311F08E9801C093
:1045E0008E9A3196EAB9FBB908C082B1882311F0DE
:1045F0008E9801C08E9A8FEF82B924B135B186B101
:1046000097B12817390711F48AE00FC0E8B1F9B162
:10461000CF01019688B999B9818180B986E005C03A
:104620008E988BE002C08E988CE081B90BC01092FE
:10463000000A1092060A109240081092410881E088
:104640008093AB29FF91EF919F918F913F912F9193
:104650000F900BBE0F9008BE0F900FBE0F901F90D3
:104660001895CF93DF93EAEAF9E210821182E0E431
:10467000F6E0128A84E08283C0E8D1E082E68E838D
:10468000A0E2B6E081E016968C93169711968C9373
:10469000119796E012969C93129751968C9351978E
:1046A00042E052964C9352971A961C921A9733E016
:1046B00019963C9399E598839AE5998390E49183C0
:1046C0009683A0EBB0E012962C911297207F129661
:1046D0002C93129712962C911297226012962C937B
:1046E00020E321832683908B868345833183E0E01A
:1046F000F8E083E1818321E030E026A337A320A7FF
:1047000031A7E0E8F8E014868083E0E2F3E013826A
:10471000118288E0828391E1908320911E20309164
:104720001F20208F318FE0E8F3E09CE392838083A9
:1047300093838183DF91CF91D8CDA0E2B6E01A9622
:104740001C921A97EAEAF9E210821182E0E0F9E09D
:1047500010821382178280E18487E0E0FAE0108201
:104760001382168281E08487E0E4F8E010821182EF
:1047700016968C938E980895CF93DF938091AA29F3
:10478000882309F47EC01092AA29C6B1D7B1C730D8
:10479000D10508F471C0AE01495F5F4F93E05695B3
:1047A00047959A95E1F7E091552BF091562B6AEADF
:1047B0007DE280E41995E091582BF091592B878187
:1047C000883019F483E180938C298681883019F42C
:1047D00083E180938B29E0914B2BF0914C2BBE0110
:1047E0008AEA9DE21995EC0194FF06C0DF7E8AE219
:1047F0009EE28AB99BB902C01AB81BB82097E1F1B2
:10480000AE01495F5F4F83E0569547958A95E1F782
:10481000E091552BF091562B6AEA7DE281E41995DF
:10482000E091582BF091592B8781893019F483E15D
:1048300080938C298681893019F483E180938B29B8
:10484000C6B9D7B98AEA9DE288B999B910926008C9
:10485000109261088FE090E080936608909367085B
:1048600088E090E080936A0890936B0883E28093DD
:10487000410883E081B905C01092000A1092060A2F
:1048800034DD8091AB29882329F01092AB29DF9188
:10489000CF912BCDDF91CF910895CF93DF93E0E4BB
:1048A000F6E0128A84E08283C0E8D1E082E68E835B
:1048B000A0E2B6E081E016968C93169711968C9341
:1048C000119796E012969C93129751968C9351975C
:1048D00042E052964C9352971A961C921A9733E0E4
:1048E00019963C93199799E598839AE5998390E4F2
:1048F00091839683C0EBD0E02A81207F2A832A818E
:1049000022602A8320E321832683908B868345833C
:104910003183E0E0F8E093E1918321E030E026A3E9
:1049200037A320A731A7E0E8F8E014869083E0E2FF
:10493000F3E01382118298E0928341E14083409139
:104940001E2050911F20408F518FE0E8F3E04CE390
:10495000428390834383918315968C93E0E0F9E042
:104960008FE790E086A397A322A733A71082168231
:104970008CE087831092000A1092AC29EFEAF9E2EA
:10498000108212821182DF91CF91089581E080938D
:1049900026067EDCE0E0F9E010821782E0E0FAE033
:1049A00010821782EFEAF9E21182128210820895D2
:1049B0001F920F920FB60F92112408B60F9218BED5
:1049C0000BB60F921BBE2F933F938F939F93EF9342
:1049D000FF93E091AC29F0E0EE0FFF1FE25CFF4D8A
:1049E0000190F081E02D199410928C08109200082B
:1049F00086E18A95F1F700C081E08093000883E0AA
:104A000080938C0818B88091AA2D86B917B882E0D7
:104A100001C083E08093AC2986C0309911C082B177
:104A200081110EC010928C081092000896E19A95A0
:104A3000F1F700C081E08093000883E080938C0848
:104A400084E0E8CF309B10C010928C0810920008D0
:104A500086E18A95F1F700C081E08093000893E039
:104A600090938C0882B901C012B886B1869586B938
:104A700084B195B1019784B995B9892B11F485E07A
:104A800001C083E08093AC2987B18F5F87B98770BD
:104A900009F049C0E8B1EF5FE8B9F0E0E655F24D42
:104AA000808186B940C082B181110EC010928C08FD
:104AB0001092000896E19A95F1F700C081E080938A
:104AC000000883E080938C0886E0A4CF1092000950
:104AD00082E591E00197F1F700C0000082E0809349
:104AE000870389E3809381038AEA9DE28AB99BB9AF
:104AF00081E090E084B995B980E886B98EB19FB124
:104B00002091080430910904822B932B8093AD29C6
:104B10009093AE2981E08093B12918B817B810920C
:104B2000AC2901C000C0FF91EF919F918F913F91FF
:104B30002F910F900BBE0F9008BE0F900FBE0F90DD
:104B40001F9018951F920F920FB60F92112408B65E
:104B50000F9218BE0BB60F921BBE2F933F934F932D
:104B60005F938F939F93EF93FF931092070A109296
:104B7000000A1092470910924009809181038E7FAC
:104B80008093810384B195B187709927892BC9F0EF
:104B9000E4B1F5B186B144B155B193E0F695E7952E
:104BA0009A95E1F7E655F24D90E04770552728E0D9
:104BB00030E0241B350B02C0959587952A95E2F7C6
:104BC000808381E08093B0291092B1298FEF9FEF0D
:104BD0008093260A9093270A1092200A1092210AA5
:104BE0001092060A1092070A1092030A84E080933A
:104BF000000A87E08093AC29FF91EF919F918F91FC
:104C00005F914F913F912F910F900BBE0F9008BE77
:104C10000F900FBE0F901F9018951F920F920FB616
:104C20000F92112408B60F9218BE0BB60F921BBE3E
:104C30008F93EF93FF93E0E8F3E081818F7C818392
:104C4000E0E0FAE088E8838381E08083FF91EF91E0
:104C50008F910F900BBE0F9008BE0F900FBE0F905C
:104C60001F9018951F920F920FB60F92112408B63D
:104C70000F9218BE0BB60F921BBE2F933F934F930C
:104C80005F938F939F93EF93FF93809160091092AE
:104C900060091092610992E090934009813620F0FA
:104CA000813A08F063C077C086B1869586B984B131
:104CB00095B1019684B995B987709927892B41F4EC
:104CC000EAB1FBB1CF0101968AB99BB986B1808365
:104CD00084B195B180FD88C0369986C01092070ACC
:104CE0001092000A109247091092400980918103A6
:104CF0008E7F8093810384B195B187709927892B2A
:104D0000C9F0E4B1F5B186B144B155B193E0F6957F
:104D1000E7959A95E1F7E655F24D90E047705527F3
:104D200028E030E0241B350B02C0959587952A9525
:104D3000E2F7808381E08093B0291092B1298FEF50
:104D40009FEF8093260A9093270A1092200A1092D0
:104D5000210A1092060A1092070A1092030A84E0B0
:104D60008093000A87E08093AC293EC086B1869587
:104D7000806886B984B195B1019684B995B9877078
:104D80009927892B41F4EAB1FBB1CF0101968AB989
:104D90009BB986B1808386B18695806886B984B1D7
:104DA00095B1019684B995B987709927892B41F4FB
:104DB000EAB1FBB1CF0101968AB99BB986B1808374
:104DC00086B1869586B984B195B1019684B995B9B5
:104DD00087709927892B41F4EAB1FBB1CF01019685
:104DE0008AB99BB986B18083FF91EF919F918F9192
:104DF0005F914F913F912F910F900BBE0F9008BE86
:104E00000F900FBE0F901F901895BF92CF92DF9218
:104E1000EF92FF920F931F93CF93DF93CDB7DEB73F
:104E2000DA95CDBFDEBF8091B1298823B9F08EB16C
:104E30009FB140910804509109042091AD2930910F
:104E4000AE29842B952B821B930B039738F014B853
:104E500015B881E08093B0291092B12922DA882315
:104E600009F440C18091B12981113CC18091AF29E1
:104E7000811105C08091B029882309F433C1809144
:104E8000AC29873041F48091200A9091210A853223
:104E9000914008F427C18091B029882309F4A6C065
:104EA00084B195B1892B09F4A1C084B195B108975B
:104EB00018F414B815B89AC044B155B1495F5F4FA2
:104EC00063E0569547956A95E1F76AEA7DE2CE017F
:104ED00001960E94D6458AEA9DE28AB99BB904B13F
:104EE00015B114B815B8C12CD12C73E1B72EE8E078
:104EF000EE2EF12CC016D10608F078C0F60153E072
:104F0000F695E7955A95E1F741E050E04C0F5D1FAB
:104F1000E40FF51F8081982F969596959083837066
:104F2000813039F0E8F0823009F059C086B18695B9
:104F300003C086B18695806886B984B195B1019623
:104F400084B995B987709927892B09F048C0EAB1CF
:104F5000FBB1CF0101968AB99BB986B180833FC06E
:104F600084B195B187709927892BC1F0E4B1F5B16F
:104F700086B124B135B143E0F695E7954A95E1F75E
:104F8000E655F24D90E027703327A701421B530BE3
:104F900002C0959587954A95E2F78083E091582B5A
:104FA000F091592B8781883011F4B0928C29868139
:104FB000883011F4B0928B2944B155B1495F5F4FED
:104FC00093E0569547959A95E1F7E091552BF0912E
:104FD000562B6AEA7DE280E4199581E001C080E009
:104FE00052E0C50ED11C882309F484CF1092AF295A
:104FF0001092B02964B175B1E0914B2BF0914C2B1C
:105000008AEA9DE2199584B995B984B195B1892B45
:1050100009F468C089E0809381031092000A10921D
:10502000200A1092210A8FE790E08093260A90933D
:10503000270A8FE590E08093280A9093290A10921E
:10504000060A80E180930C0A93E09093070A10927D
:105050006009109261092FEF3FEF209366093093AA
:10506000670920E031E020936809309369091092C4
:10507000460980934C0981E08093470981E1809340
:105080008001109288011092800310922906E0910D
:10509000582BF091592B8781893019F483E1809343
:1050A0008C298681893019F483E180938B2944B15E
:1050B00055B1495F5F4F83E0569547958A95E1F773
:1050C000E091552BF091562B6AEA7DE281E4199527
:1050D00081E08093AC2912B8109220091092210926
:1050E00080930009D395CDBFDEBFDF91CF911F9193
:1050F0000F91FF90EF90DF90CF90BF90089514B87C
:1051000015B881E08093AF29A4C81092070A1092C5
:10511000000A1092470910924009809181038E7F06
:105120008093810384B195B187709927892BC9F049
:10513000E4B1F5B186B144B155B193E0F695E79588
:105140009A95E1F7E655F24D90E04770552728E033
:1051500030E0241B350B02C0959587952A95E2F720
:10516000808381E08093B0291092B1298FEF9FEF67
:105170008093260A9093270A1092200A1092210AFF
:105180001092060A1092070A1092030A84E0809394
:10519000000A87E08093AC291092AC291092B029C4
:1051A0001092AF2975C881E08093B4291092B2297A
:1051B000089581E08093B42908950895CF92DF92F5
:1051C000EF92FF920F931F93CF93DF93CDB7DEB78C
:1051D0002597CDBFDEBF8C01FC0180819091B42961
:1051E0009230F1F038F0943079F120F1953009F4F3
:1051F0004AC049C121E09227292F21702093B2296A
:10520000911102C0863219F0823509F03CC184E464
:10521000F8018083118282E08093B42980E134C157
:105220009091B229911102C08632B1F0823509F015
:105230004DC012C09091B229911102C0863261F026
:10524000823509F075C008C09091B229911102C051
:10525000863211F0823539F484E4F80180831182BA
:1052600081E089270DC0803309F41BC1823A09F41B
:1052700034C1803A09F450C1803509F4F6C081E0A8
:105280008093B42900C160E170E0C8010E946132DE
:105290008823A1F08091542B81110BC06091B32918
:1052A000F4E06F9FB001112444E050E0C8010E9477
:1052B0009D0E84E08093B4298AE004C084E080934A
:1052C000B42981E0F801808384E0DEC08339B9F637
:1052D00019821A821B821C8288E8898343E050E08D
:1052E00060E070E0CE0102960E944F0EF8018181CD
:1052F000803209F4ABC0803709F048C0F8019281D0
:1053000089819813C0C093818A819813BCC094810D
:105310008B819813B8C095818C819813B4C084E0B8
:10532000808361E070E0C8010E94363283E02AC0C9
:10533000853909F0A4CF44E050E064E070E0CE018C
:1053400001960E944F0EF8018181803209F47EC0DF
:105350008037E1F4F80192818981981394C0938198
:105360008A81981390C094818B8198138CC0958109
:105370008C81981388C0108261E070E0C8010E949F
:10538000363284E08093B42988E17EC0E82EE2942E
:105390009FE0E9222EEF2E0D8F70F82E88E090E02E
:1053A0008F1991094FEF50E06A0102C0D594C7945C
:1053B0008A95E2F7253021F0243059F5FF20E9F0F5
:1053C00044E050E0B8016E5F7F4FCE0101962D831F
:1053D0000E94C9452D81892B61F49A818981892791
:1053E0009B8189279C818927F801968189278C21B7
:1053F00069F1243071F4F11046C044E050E0B80186
:105400006E5F7F4FCE0101960E94C945892BF1F056
:105410003AC02430C0F5E22EF12CA701B8016E5F2E
:105420007F4FCE0101960E94C945892B61F5D801B5
:10543000AE0DBF1DE1E0F0E0EC0FFD1FEE0DFF1D16
:1054400012969C9180818927C822E9F42981F8016C
:1054500020833A8131839B8192838C8183832327AC
:1054600092278927848388E20FC0F8018181811106
:1054700041C062E070E0C8010E946132882309F4F3
:1054800020CF1092B42980E090E02596CDBFDEBFFA
:10549000DF91CF911F910F91FF90EF90DF90CF9010
:1054A0000895F801F18062E070E0C8010E94613265
:1054B000882309F406CFFFE0FF15E0F084E0F89EB2
:1054C000B001112440E150E0C8010E944F0E60E19C
:1054D00070E0C801CBD780E9D7CFF801F18066E052
:1054E00070E0C801EED7882309F4EBCE8EEF8F0D64
:1054F0008E3018F0F8011082E7CE8091542B811184
:10550000DBCEF4E0FF9EB001112444E050E0C8017E
:1055100002960E949D0ED0CEF801F18062E070E00C
:10552000C801CFD7882309F4CCCE8EEF8F0D8E30F3
:1055300008F7F092B32985E0BDCECF93DF93EC015D
:1055400043E050E060E070E00E944F0E44E050E025
:1055500064E070E0CE010396DF91CF910C944F0E82
:105560000F931F93CF93DF931F921F92CDB7DEB798
:105570008C01FC0190818181892798E8892792819B
:1055800089278A83948183818927958189279681B8
:105590008927898343E050E060E070E0C8010E9401
:1055A0009D0E41E050E063E070E0CE0102960E9463
:1055B0009D0E44E050E064E070E0C80103960E9454
:1055C0009D0E41E050E068E070E0CE0101960E943F
:1055D0009D0E0F900F90DF91CF911F910F91089525
:1055E00081E08093D22984E090E08093B729909362
:1055F000B82988E08093B6291092B529089581E0F2
:105600008093D22982E490E08093B7299093B829BF
:1056100088E18093B6291092B529089581E080939E
:10562000D229089508958F929F92AF92BF92CF9200
:10563000DF92EF92FF920F931F93CF93DF93CDB73B
:10564000DEB72F97CDBFDEBF8C016B018091D229D1
:10565000853009F4C1C058F4823009F446C050F1D5
:10566000833009F48BC0843009F4A6C0EBC58830C0
:1056700009F45BC198F4863009F4C2C0873009F0A0
:10568000E1C5C8010E947F336801F4E0CF0ED11C50
:105690007601580128E0A20EB11CE4C0893009F45B
:1056A000DCC28D3008F0CEC578016801B6E0CB0EC3
:1056B000D11C10C391E08927982F91709093B52940
:1056C0003091B7292091B829D8019C91811102C04D
:1056D000963219F0923509F0BDC3F8013083218369
:1056E00084E08093D22980E1AEC5F8018081982FB3
:1056F0009D7F913411F48AE085C2803329F562E000
:1057000070E0C801DED68823E9F0D80111966C91CB
:10571000B0E16B9FB001112440E150E0C8010E944C
:105720004F0E60E170E0C801A1D680E98CC590EA17
:10573000980F923008F006C662E070E0C801C1D64A
:10574000811183C581E05DC2803A91F462E070E02E
:10575000C801B7D68823B1F3D80111968C9111975F
:105760008093C92983E08093D2298AE08C93B0C2C8
:10577000803509F067C5F80181815CC060E170E0A7
:10578000C8019FD6882399F08091542B81110BC0BA
:105790006091C929B0E16B9FB001112440E150E054
:1057A000C8010E949D0E8AE0F801808303C081E059
:1057B000D8018C9382E08AC29091B5293091B729A3
:1057C0002091B829F8018081911102C0863299F0A8
:1057D000823509F047C30FC09091B5293091B729A0
:1057E0002091B829F8018081911102C0863219F008
:1057F000823509F072C4D8013C9311962C9311C0E4
:105800009091B5293091B7292091B829D8018C9170
:10581000911102C0863211F0823531F4F8013083E3
:10582000218381E0892708C3803509F080CFD80122
:1058300011968C91882319F0D8011C9249C262E01C
:1058400070E0C8013ED6882309F47CCFE091552B47
:10585000F091562B40E060E070E081E919951092DC
:10586000D229F0C471D7D7019C918927F701819380
:105870007F01EA15FB05B1F7E091552BF091562B0E
:1058800044E0B60180EA1995D80114969C911497CA
:105890008091CA29981340C015969C9115978091C4
:1058A000CB29981339C016969C9116978091CC29D4
:1058B000981332C017969C918091CD2998132CC0D3
:1058C00068018EECA82E89E2B82E94E0E92EEA0C4D
:1058D0004501F501F1905F0137D78F25D6018D93F2
:1058E0006D01D401EC91F0E0EC59FB4FF4905ED6E1
:1058F000D601A158BF4F8F258C93EA10E9CFE091D4
:10590000552BF091562B44E0B80181EA199588E0B7
:105910008093D22980E256C0E091552BF091562B0E
:1059200040E060E070E080EC95C178014801B4E0AF
:105930008B0E911C580108D7F50190818927D5015C
:105940008D935D01A815B905B1F7F8018081803309
:1059500009F048C062E070E0C801B3D58823A1F126
:10596000D80111966C91B0E16B9FB001112440E118
:1059700050E0C8010E944F0E60E170E0C80176D58A
:10598000E091552BF091562B42E1B80180E8199532
:105990006801E2E1CE0ED11CD7011C91D5D681273A
:1059A000F70181937F01E12FF0E0EC59FB4F149157
:1059B000FDD5D701A158BF4F81278C93EC14FD046E
:1059C00059F780E990E1FDC4D2D691E08927D8014A
:1059D0008C93E091552BF091562B44E0B80181EC6B
:1059E000199576C1803A71F462E070E0C80169D51A
:1059F000882351F1F80181818093C92989E080933E
:105A0000D22967C0803C69F462E070E0C80159D5D2
:105A10008823A1F1D80111968C918093C9298BE03C
:105A200028C0813CC1F462E070E0C8014AD58823F7
:105A300059F0F80181818093C929BAE0FB2EF092D8
:105A4000D22995D68F2548C0E091552BF091562B41
:105A500044E0B80143C0823CE1F462E070E0C80178
:105A600030D5882359F0D80111968C918093C9299B
:105A70008CE08093D2297BD69AE0C2C0E091552B6E
:105A8000F091562B44E0B80181EC199570D691E065
:105A900022C0803B31F562E070E0C80112D5E09190
:105AA000552BF091562B44E0B8018823B9F086E8D5
:105AB00019958091542B81110CC0F8016181F0E19E
:105AC0006F9FB001112440E150E089EB99E20E9400
:105AD0009D0E4DD69AE08927D80148CE81EC1995C4
:105AE0008DC090EA980F923008F08EC062E070E0AE
:105AF000C801E7D4882309F481C0D80111962C91FC
:105B00001197322F3C7F8C91803619F08AE390E018
:105B100002C080E390E06C01B0E13B9FC00CD11C5F
:105B2000112427FF0AC0207FE0E12E9F800D911DE8
:105B300011249C0120543F4F6901E091552BF091B5
:105B4000562B42E0B80180E9199564E0CE01079632
:105B50000E948D0D8091532B44E050E0873019F462
:105B600063E070E002C060E070E0CE010B960E943E
:105B70004F0E46E050E0B601CE0101960E944F0E56
:105B80008F818093CA2988858093CB2989858093CA
:105B9000CC298A858093CD2960E470E08AEC99E273
:105BA000F9D58091CA298093CE298091CB29809301
:105BB000CF298091CC298093D0298091CD298093C1
:105BC000D12960E270E08EEC99E2E4D5AE01495F44
:105BD0005F4FBE01655F7F4FCE01019620D5FE016C
:105BE000379684E08E0F9191D7019D937D018E139E
:105BF000FACF87E08093D22980E225C3B8D591E01F
:105C00008927F801808364C08035B1F481818111D6
:105C100013CE62E070E0C80154D4882309F492CD19
:105C20001092D229E091552BF091562B40E060E084
:105C300070E081E9199506C3A601495F5F4FA3E0B3
:105C400056954795AA95E1F7E091552BF091562B83
:105C5000B80182E9199581E0EFC078016801B2E1ED
:105C6000CB0ED11C71D5F70190818927D7018D9377
:105C70007D01AC15BD05B1F760E170E0C80121D42C
:105C8000E091552BF091562B8823B1F042E1B801F9
:105C900081E819958091542B81110BC06091C9291D
:105CA000B0E16B9FB001112440E150E0C8010E94B7
:105CB0009D0E5DD59AE081C344E0B80181EC199551
:105CC00056D591E08927D8018C9388E08093D2291A
:105CD00084E0B9C239D5F70190818927D7018D9326
:105CE0007D01AC15BD05B1F764E070E0C801E9D3F2
:105CF000882309F4A4C06091C929B0E16B9FB00169
:105D0000112440E150E089EB99E20E944F0E9091FE
:105D1000B9298091BD29809598134DC38091C129DF
:105D2000981349C32091BA298091BE2980952813E0
:105D300042C38091C22928133EC3C090BB298091E1
:105D4000BF298095C81237C38091C329C81233C3B5
:105D50008091BC293091C029309583132CC3309198
:105D6000C429831328C34091C5293091C629309591
:105D7000431321C33091C72943131DC33091C82950
:105D80003095431318C3D8013C9111964C9111974B
:105D900012968C901297912CA12CB12C540199241D
:105DA0008824942A832A13963C91B32AD12CE12C7F
:105DB000F12C7601DD24CC24D22AC92AF82A80913C
:105DC000D2298B3009F0DCC2E091552BF091562B93
:105DD00046E0B80185E81995C818D908EA08FB0813
:105DE000C092B92933272F2D1E2D0D2D0093BA29CE
:105DF000A701662777274093BB298F2D9927AA27CC
:105E0000BB278093BC29EC2DE095E093BD29E02FC2
:105E1000E095E093BE29E42FE095E093BF29E82FB9
:105E2000E095E093C029C092C1290093C229409314
:105E3000C3298093C42988E08093D22903C2E091CA
:105E4000552BF091562B44E0B80181EC19958FD475
:105E500091E0B3C2903409F0F5C182E08093D22979
:105E60008AE03ACE833909F0FACC8091532B8730FF
:105E700009F0A1C043E050E060E070E0CE0102967E
:105E80000E944F0E88E88983F8019181903219F0C1
:105E9000903761F024C0D80180833A8131832B810F
:105EA00022839C8193832327822739C1F801828131
:105EB000883809F0C7C193818A819813C3C194813E
:105EC0008B819813BFC195818C819813BBC184E0ED
:105ED000808361E070E0C801C9D285E03DC1E92E50
:105EE000E2944FE0E4222EEF2E0D9F70F92E88E011
:105EF00090E08F1991094FEF50E06A0102C0D594EC
:105F0000C7948A95E2F7253021F0243061F5FF200F
:105F1000F1F044E050E0B8016E5F7F4FCE01019692
:105F20002F870E94C9452F85892B69F49A818B811F
:105F3000892798E889279C818927D80116969C9102
:105F400089278C2181F1243071F4F1107BC144E068
:105F500050E0B8016E5F7F4FCE0101960E94C945A7
:105F6000892B09F16FC1243008F06CC1E22EF12CAD
:105F7000A701B8016E5F7F4FCE0101960E94C9450F
:105F8000892B09F05FC1D801AE0DBF1DE1E0F0E043
:105F9000EC0FFD1FEE0DFF1D12969C91808189274D
:105FA000C82209F04FC198E8F80190833A81318303
:105FB0002B8122830CC144E050E060E070E0CE0110
:105FC00001960E944F0E9091B629D80111968C919E
:105FD000803209F4F5C08037D9F4D80112962C919B
:105FE0001297898128132EC113962C9113978A81B9
:105FF000281328C114962C9114978B81281322C141
:1060000015962C9115978C8128131CC19C939FC0C9
:10601000E82EE2943FE0E3222EEF2E0D8F70F82E53
:1060200088E090E08F1991094FEF50E06A0102C0BB
:10603000D594C7948A95E2F7253021F0243061F594
:10604000FF20F1F044E050E0B8016E5F7F4FCE01D9
:1060500001962F870E94C9452F85892B69F49A8163
:10606000898189279B8189279C818927F8019681CD
:1060700089278C2109F442C0243071F4F110E2C068
:1060800044E050E0B8016E5F7F4FCE0101960E9460
:10609000C945892B99F1D6C0243008F0D3C0E22E2F
:1060A000F12CA701B8016E5F7F4FCE0101960E94CF
:1060B000C945892B09F0C6C0D801AE0DBF1DE1E06E
:1060C000F0E0EC0FFD1FEE0DFF1D12969C918081FC
:1060D0008927C82209F0B6C011C0853909F0BFCBA5
:1060E00044E050E063E070E0CE0101960E944F0E64
:1060F0009091B629F80181818032A9F42981D801D3
:106100002C933A8111963C9311979B8112969C9304
:1061100012978C8113968C931397232792278927A4
:1061200014968C935AC08037D9F4F8012281898162
:10613000281388C023818A81281384C024818B81FD
:10614000281380C025818C8128137CC0908361E056
:1061500070E0C8018BD186E08093D22988E173C0BA
:10616000E82EE2942FE0E2222EEF2E0D8F70F82E13
:1061700088E090E08F1991094FEF50E06A0102C06A
:10618000D594C7948A95E2F7253049F544E050E06C
:10619000B8016E5F7F4FCE0101962F870E94C945DF
:1061A0002F85892B09F59A81898189279B818927E8
:1061B0009C818927D80116969C9189278C21A1F46E
:1061C0002981F80120833A8131839B8192838C81DC
:1061D0008383232792278927848388E234C024304D
:1061E00099F4FF2029F0D2CF243071F4F1102AC0A5
:1061F00044E050E0B8016E5F7F4FCE0101960E94EF
:10620000C945892BE9F21EC02430E0F4E22EF12CBE
:10621000A701B8016E5F7F4FCE0101960E94C9456C
:10622000892B81F4D801AE0DBF1DE1E0F0E0EC0F49
:10623000FD1FEE0DFF1D12969C9180818927C822BB
:1062400009F4BECF80E090E0BCC0F8012181322F7C
:106250003C7F8081803619F08AE390E002C080E3C1
:1062600090E06C01F0E13F9FC00CD11C112427FF8E
:106270000AC0207F30E1239F800D911D1124DC0195
:10628000A054BF4F6D01E091552BF091562B42E089
:10629000B80180E919957E01B7E0EB0EF11C64E0CE
:1062A000C7010E948D0D8091532B44E050E0873050
:1062B00019F463E070E002C060E070E0CE010B967C
:1062C0000E944F0E46E050E0B601CE0101960E94BA
:1062D0004F0E8F818093CA2988858093CB29898529
:1062E0008093CC298A858093CD2960E470E08AEC84
:1062F00099E250D28091CA298093CE298091CB29EE
:106300008093CF298091CC298093D0298091CD2969
:106310008093D12960E270E08EEC99E23BD287E075
:106320008093D229D801F70184E08E0D91919D933D
:106330008E13FCCFA701BE01655F7F4FCE01019692
:106340006ED15ACC982F9F77903329F0803A19F06C
:10635000805C833078F481E08093D22984E0F80176
:106360008083E091552BF091562B40E060E070E087
:1063700082EC36CBE091552BF091562B40E068CC67
:106380008A3069F4E091552BF091562B46E0B80124
:1063900084E81995C80CD91CEA1CFB1C21CD8C3053
:1063A00009F01ECDE091552BF091562B46E0B80137
:1063B00087E8199515CDDBD196E08927F801808310
:1063C00084CC2F96CDBFDEBFDF91CF911F910F916F
:1063D000FF90EF90DF90CF90BF90AF909F908F9005
:1063E0000895CF93DF932091532B273071F4EC0164
:1063F00043E050E060E070E00E944F0E44E050E067
:1064000063E070E0CE01039604C044E050E060E039
:1064100070E0DF91CF910C944F0ECF93DF931F92DA
:10642000CDB7DEB72091532B273029F447E050E059
:1064300060E070E015C0FC013181208123273281AA
:10644000232733812327298344E050E060E070E074
:106450000E949D0E41E050E064E070E0CE010196A4
:106460000E949D0E0F90DF91CF91089520E420931C
:10647000D00026EC2093D5002093D40021E0209377
:10648000D000DC01680F791FA617B70741F0ED9126
:10649000F0E0EC59FA4FE491E093D300F5CFE091AE
:1064A000D500F0E0EC59FA4FE491EC93E091D40080
:1064B000F0E0EC59FA4FE4911196EC931092D00071
:1064C000089520E42093D00026EC2093D50020935B
:1064D000D40021E02093D000DC01680F791FA617BB
:1064E000B70741F0ED91F0E0EC59FA4FE491E093F9
:1064F000D300F5CFE091D500F0E0EC59FA4FE491EC
:106500008C918E130AC0E091D400F0E0EC59FA4F60
:10651000E49181E011969C919E1380E01092D0004E
:1065200081700895F091D629A091D7294091D8295A
:10653000E091D3293091D4292091D5295A2F507137
:106540009F2F917E9527542F507295275E2F547957
:106550009527532F53779527522F5A739527592FE5
:1065600052955F709527592F569556959527B92FB7
:10657000B69550E060E070E0BA01552744275A2BE9
:106580004F2B76956795579547959B279170981354
:106590006068E093D6293093D7292093D829409377
:1065A000D3295093D4296093D5290895CF93DF93AD
:1065B00083ED99E2DC011196EC911197CE2FCF700B
:1065C000D0E0C259DF4D2C91A22FA295AF70B0E060
:1065D000A259BF4D38892C91232BE295EF70F0E042
:1065E000E259FF4D30A1232BDC011296EC91AE2F26
:1065F000AF70B0E0A259BF4DD0968C91922F982BDE
:10660000E295EF70F0E0E255FF4D8081E92FE82B35
:10661000F0E0E25BFF4D8081DF91CF910895CF9252
:10662000DF92EF92FF920F931F93CF93DF93FB01C3
:10663000EA01BC016F5F7F4F03ED19E2B6EDEB2E6F
:10664000B9E2FB2E53E05E0DCB010197DC012C91EA
:10665000DB018C9130E0382B88E090E040E04695FB
:10666000969520FD406821FD9068369527953695D2
:1066700027958150A1F7D7014D937D01D8019D93B6
:106680008D016E5F7F4F5E11DFCF918189819827E9
:10669000C2808A81C826D12CE12CF12C7601DD2420
:1066A000CC24D92A908188818927C82A93818B811B
:1066B0008927F82A10E27ADF082F8C2D817032DFCB
:1066C000F694E794D794C794002311F06894F7F8F0
:1066D000115089F788818C25888389818D2589834C
:1066E0008A818E258A838B818F258B83DF91CF9141
:1066F0001F910F91FF90EF90DF90CF900895CF9270
:10670000DF92EF92FF92CF93FC018181C280D12C66
:10671000E12CF12C7601DD24CC24D82A8081C82AF2
:106720008381F82AC0E242DF9C2D91708927FADE2E
:10673000F694E794D794C794C150A9F7CF91FF90EE
:10674000EF90DF90CF9008951F93CF93DF93D8E021
:10675000C0E02CDF182F80E0E5DEC6951111C0687F
:10676000D150B9F78C2FDF91CF911F9108951F93CE
:10677000CF93DF93D4E0C0E019DF182F80E0D2DEA2
:10678000C6951111C860D150B9F78C2FDF91CF9108
:106790001F910895FC01CB01019728F14281242F1C
:1067A0002D72322F32953F702327322F3695369532
:1067B0002327322F3695A18150E060E070E0BA01C6
:1067C000552744275A2BA0814A2BA3817A2B7695F3
:1067D000679557954795232720FD7068408351831F
:1067E00062837383D9CF0895AF92BF92CF92DF9225
:1067F000EF92FF920F931F93CF93DF936730710552
:1068000009F451C09B0127703327232B09F04EC098
:10681000EB016C015B0183E0B694A7948A95E1F7E4
:106820007B0196E0F694E7949A95E1F7EA0CFB1C5D
:10683000EC0CFD1C8501015011090C0D1D1DA7015B
:10684000401B510B60E070E0C80101960E94F045CA
:106850000C151D0520F1D801EC91F0E0EC59FB4F2F
:1068600044919701D7010A171B0768F48C91982F60
:10687000990FF90182919F01881F8827881F892B12
:106880008C931197F0CF11968C9111978E7FE42FF6
:10689000E170E82B1196EC9301501109D9CFC50195
:1068A0008C0F9D1F04C087E090E001C0CB01DF91F9
:1068B000CF911F910F91FF90EF90DF90CF90BF90FD
:1068C000AF900895EF92FF920F931F93CF93DF93B2
:1068D000EC01CB0167307105D1F169E070E00E94F5
:1068E0002045DE0120E030E088E090E02617370701
:1068F00039F1F90143E0F695E7954A95E1F7E20FA2
:10690000F31FEC0FFD1F408150E089010770112734
:10691000002E02C0559547950A94E2F74C93011555
:10692000110551F0E1817C01E01AF10A01C0EE0F7E
:10693000EA94EAF74E2B4C932F5F3F4F1196D6CF38
:10694000C90123E0880F991F2A95E1F702C087E06B
:1069500090E0DF91CF911F910F91FF90EF900895FC
:10696000CF93DF93FC016115710511F1808186954C
:1069700080839B01295F3F4F83E0369527958A9559
:10698000E1F7DF0141E050E04217530770F4C19195
:106990009081D0E89D9FC00111248C2B8D93808124
:1069A000869580834F5F5F4FEFCFCB01019702C089
:1069B00080E090E0DF91CF910895EF92FF920F93E6
:1069C0001F93CF93DF93EC01CB016730710509F47E
:1069D00042C069E070E00E94204520E030E088E09D
:1069E00090E026173707B9F1D90143E0B695A7958E
:1069F0004A95E1F7A20FB31FA90147705527AC0FC5
:106A0000BD1FEC91F0E0042E02C0F595E7950A94C5
:106A1000E2F74115510559F011960C9111977C013F
:106A2000E41AF50A01C0000FEA94EAF7E02BF0E05F
:106A3000EC59FB4FE4911196AC91B0E08D0102C08E
:106A4000159507954A95E2F7A8014E2740FD05C028
:106A50002F5F3F4FC6CF81E001C080E0DF91CF9133
:106A60001F910F91FF90EF9008951092392A089589
:106A70001092392A1092D92910923A2A0895F8DFF3
:106A80000E9485281092392A089508950895DC01FE
:106A900023E633E66150E8F04D91942F922780E190
:106AA000989FA00111244927E42FF0E042954F70F0
:106AB000232F3327C9018427AC013E2F2227242707
:106AC000352743E0EE0FFF1F4A95E1F72E273F27BA
:106AD000E1CFC90108958F929F92AF92BF92CF925A
:106AE000DF92EF92FF920F931F93CF93DF93CDB777
:106AF000DEB7C154D240CDBFDEBF8C016B01209107
:106B0000D929233009F43DC138F4213069F022300D
:106B100009F4B3C00C94AD3D243009F4B1C2253062
:106B200009F4CFC40C94AD3DE0903B2BF0903C2B8E
:106B3000E114F104B9F0A701495F5F4F23E05695D6
:106B400047952A95E1F76BE37AE20E94D64560917A
:106B50003B2B70913C2BC80147DE10923B2B1092CF
:106B60003C2BADC46115710509F4A8C0F9DE5C01C8
:106B7000BC01C80122DFD82EB501C801A3DE5C012B
:106B80009C01295F3F4FA901440F551F93E0569583
:106B900047959A95E1F74A5F5F4F4138510538F0C4
:106BA00062EC70E2CE0101960E94024690C0A3E022
:106BB00036952795AA95E1F7A80160E870E0CE0127
:106BC00001960E94A60D8C01CF5FDD4FB882C150A7
:106BD000D240CE5FDD4FA882C250D24085E691E21E
:106BE0009F938F93B0E8AB2EB12CC501801B910B06
:106BF0009F938F9381E090E08C0F9D1F800F911FDA
:106C00009F938F930E940946080F191FB501601BBF
:106C1000710B22E030E0AE014F5F5D4F81E090E00C
:106C20008C0F9D1F800F911F0E94A60D800F911F3A
:106C30000F900F900F900F900F900F90A501481B91
:106C4000590B21E030E02C0F3D1F280F391FD110C8
:106C500003C081ED90E202C080EE90E29F938F939B
:106C60005F934F933F932F930E9409460F900F908D
:106C70000F900F900F900F902AC0E0903B2BF09058
:106C80003C2BE114F104B9F0A701495F5F4FF3E039
:106C900056954795FA95E1F76BE37AE20E94D6455F
:106CA00090913B2B80913C2B10923B2B10923C2BD4
:106CB000E92EF82E54C76115710591F488E0EBE7D1
:106CC000F1E2DE01119601900D928A95E1F71092A2
:106CD000D929BE016F5F7F4F85E60E94B2203FC772
:106CE0009B01295F3F4F73E0369527957A95E1F731
:106CF000AC0160E870E0CE0101960E94A60D8C0107
:106D0000CF5FDD4FD882C150D240CE5FDD4FC88209
:106D1000C250D24085E691E29F938F93E0E8CE2E59
:106D2000D12CC601801B910B9F938F9381E090E043
:106D30008C0F9D1F800F911F9F938F930E94094678
:106D4000800F911FB601681B790B22E030E0AE0185
:106D50004F5F5D4FA1E0B0E0AC0FBD1F8A0F9B1FDE
:106D60000E94A60D1092D929BE016F5F7F4F85E664
:106D70000E94B2200F900F900F900F900F900F90E5
:106D8000EEC680913A2A81115CC1B090392AB5E0F3
:106D9000BB1588F0E3E0BE1608F04BC0F1E0FB1530
:106DA00098F082E5D8018C9382E08093392A67E0DD
:106DB000E62EF12C48C128E02B1508F0B8C03AE0C7
:106DC000B31609F403C13DC16331710508F4C8C0AD
:106DD000C801CF5BDD4F2883C154D240C1DD7C01A7
:106DE000BC01C801EADDCF5BDD4F2881C154D24030
:106DF000882359F1B701C801CF5BDD4F2883C15407
:106E0000D24060DDF801818190E0982F88273081A1
:106E1000832B80932B2A90932C2A83E9808380E212
:106E20008183CF5BDD4F2881C154D2402093392A22
:106E3000B9C0C80195DD7C01BC01C801BEDD882355
:106E400021F0F8E0EF16F10488F41092392AC70116
:106E5000089667E070E00E942045462FE091552B90
:106E6000F091562BB80181EC1995B6C0B701C80155
:106E700029DDD8012C9111968C91119782271296B9
:106E80009C911297892713969C91139789271496A2
:106E90009C911497891364C08B2D90E00397283838
:106EA00081F49C01220F331F820F931FFC01E25DCE
:106EB000F54D11962D913D914C9120833183428364
:106EC00012C0FC01EE0FFF1F8E0F9F1F9C01225D61
:106ED000354DF80180819181A281B381F9018083D0
:106EE0009183A283B38345E050E0B801C8010296C4
:106EF0000E94DF45F3E0BF1629F024E0B21621F02E
:106F000087E903C083E901C085E9D8018C9380E754
:106F100011968C9367E0C801BADDF80187839087EA
:106F200083E08B0D8093392A68E470E086C0693075
:106F30007105B0F0C80114DD7C01BC01C8013DDD64
:106F4000811111C0C701089667E070E00E942045DA
:106F5000462FE091552BF091562BB80181EC1995F5
:106F60001092392A39C0B701C801ACDC63E0C8010E
:106F70008EDD7C01892BA1F7D8018C9182FF15C091
:106F8000B8E0BB1691F0E6E0BE1611F087E901C04B
:106F900085E9D8018C9380E211968C93BA94BA94C7
:106FA000B092392A60E170E048C081E080933A2ACB
:106FB0008B2D90E00697B82EBB0C8B0D8C5F8093C9
:106FC000382AF801808180932D2A3DC06115710512
:106FD00031F481E08093392A0E947F2832C0C801B1
:106FE000BFDC7C01BC01C801E8DC81110FC0C70116
:106FF000089667E070E00E942045462FE091552BEF
:10700000F091562BB80181EC199508C0B701C80161
:1070100059DC63E0C8013BDD892BD9F282ECD80151
:107020008C9361E0C80133DDF80181839283B092D3
:10703000392A10923A2A68E170E0C801D5DB7C0158
:1070400002C0E12CF12C80913A2A882309F487C5EB
:107050002091382A30E04EE25AE264E170E0CE013D
:1070600001960E94A60DBE016F5F7F4F85E60E94CC
:10707000B22010923A2A1092D9290E9448216DC557
:1070800080913A2A811150C1B090392AF5E0FB1560
:1070900080F023E0B216D8F531E03B1598F082E598
:1070A000F801808382E08093392AE7E0EE2EF12C0C
:1070B0003DC188E08B1508F0A1C0AAE0BA1609F41A
:1070C000ECC032C16331710508F4B1C0C80148DCBD
:1070D0007C01BC01C80171DC882329F1B701C8011A
:1070E000F1DBD80111968C91119790E0982F8827A9
:1070F0002C91822B80932B2A90932C2A83E98C93BA
:1071000080E211968C9383E08093392AB2C0C80143
:1071100027DC7C01BC01C80150DC882321F0B8E0E9
:10712000EB16F10488F41092392AC701089667E03B
:1071300070E00E942045462FE091552BF091562B90
:10714000B80181EC1995AFC0B701C801BBDBF801EC
:107150002081818182279281892793818927948147
:10716000891365C08B2D90E00397283889F49C0122
:10717000220F331F820F931FFC01E25DF54DD801F2
:1071800011962D913D914C9120833183428312C001
:10719000FC01EE0FFF1F8E0F9F1F9C01225D354DDE
:1071A000F80180819181A281B381F901808391836B
:1071B000A283B38345E050E0B801C80102960E9463
:1071C000DF45F3E0BF1629F024E0B21621F087E98D
:1071D00003C083E901C085E9D8018C9380E711964B
:1071E0008C9367E0C80153DCF8018783908783E0C4
:1071F0008B0D8093392A68E470E092C06930710584
:10720000B0F0C801ADDB7C01BC01C801D6DB811147
:1072100011C0C701089667E070E00E942045462F24
:10722000E091552BF091562BB80181EC19951092F5
:10723000392A39C0B701C80145DB63E0C80127DC42
:107240007C01892BA1F7D8018C9182FF15C0B8E091
:10725000BB1691F0E6E0BE1611F087E901C085E9A2
:10726000D8018C9380E211968C93BA94BA94B09220
:10727000392A60E170E054C081E080933A2A8B2D76
:1072800090E00697B82EBB0C8B0D8C5F8093382A4C
:10729000F801808180932D2A49C06115710531F470
:1072A00081E08093392A0E947F283EC0C80158DBC4
:1072B0007C01BC01C80181DB81111AC0C70108969D
:1072C00067E070E00E942045462FE091552BF09139
:1072D000562BB80181EC199582ECD8018C9361E0B2
:1072E000C801D5DBF80181839283B092392A14C09A
:1072F000B701C801E7DA63E0C801C9DB892B81F275
:1073000082ECD8018C9361E0C801C1DBF801818374
:1073100092838AE08093392A10923A2A68E170E0D9
:10732000C80162DA7C0102C0E12CF12C80913A2A7A
:10733000882309F414C4F0901A2AFF20A9F1B60199
:10734000C8010EDB5C01009729F410921A2A1092F2
:107350003A2A42C0823A910540F0BC01C8012DDBB7
:1073600091E08927C82ED12C03C0CC24C394D12C02
:10737000B501C801A7DACD2829F462E1C80187DB8D
:10738000892B29F0ACEFAF0DA0931A2A2AC024E074
:10739000F29ED0011124A653B64D80E1F801019070
:1073A0000D928A95E1F71DC042E050E066E171E17F
:1073B000CE0101960E94A845E9E1F1E1E491209116
:1073C0002B2A30912C2A89819A812817390721F498
:1073D00080912D2A8E1729F01092392A0E947F2839
:1073E000BCC320911A2A203109F04DC010923A2ACC
:1073F00010921A2A1092D92920E130E04AED59E280
:1074000067E870E0CE0101960E94A60D65E671E284
:10741000CE0181960E94024620E130E04AEE59E218
:1074200065E670E0CE0183960E94A60D65E671E2E6
:10743000CE018D5B9F4F0E94024620E130E04AEF73
:1074400059E263E470E0CE018B5B9F4F0E94A60D72
:1074500065E671E2CE018B599F4F0E94024620E102
:1074600030E04AE05AE261E270E0CE0189599F4F74
:107470000E94A60D0E944821BE016F5F7F4F85E6E6
:107480000E94B2206AC380E3D8018C9311962C939A
:1074900062E0C801CF5BDD4F2883C154D240F7DAE8
:1074A000F80182839383CF5BDD4F2881C154D240A2
:1074B0002C5F20931A2A60E270E0C80195D97C0104
:1074C0004EC380913A2A811143C1B090392AF5E028
:1074D000FB1580F023E0B216C8F531E03B1598F0BB
:1074E00082E5F801808382E08093392A37E0E32E39
:1074F000F12C30C188E08B1508F09FC0AAE0BA16C5
:1075000009F4EAC025C16331710508F4AFC0C801B0
:1075100027DA7C01BC01C80150DA882319F1B701D0
:10752000C801D0D9D80111968C91119790E0982F6D
:1075300088272C91822B80932B2A90932C2A83E9E5
:107540008C9380E211968C9383E0B0C0C80108DA76
:107550007C01BC01C80131DA882321F0B8E0EB16C8
:10756000F10488F41092392AC701089667E070E0A8
:107570000E942045462FE091552BF091562BB801E3
:1075800081EC1995AFC0B701C8019CD9F8012081E1
:107590008181822792818927938189279481891308
:1075A00065C08B2D90E00397283889F49C01220F49
:1075B000331F820F931FFC01E25DF54DD801119638
:1075C0002D913D914C9120833183428312C0FC0167
:1075D000EE0FFF1F8E0F9F1F9C01225D354DF8019E
:1075E00080819181A281B381F90180839183A283FB
:1075F000B38345E050E0B801C80102960E94DF4520
:10760000F3E0BF1629F024E0B21621F087E903C0A9
:1076100083E901C085E9D8018C9380E711968C93AA
:1076200067E0C80134DAF8018783908783E08B0D27
:107630008093392A68E470E087C069307105B0F042
:10764000C8018ED97C01BC01C801B7D9811111C014
:10765000C701089667E070E00E942045462FE09140
:10766000552BF091562BB80181EC19951092392ABF
:1076700039C0B701C80126D963E0C80108DA7C0126
:10768000892BA1F7D8018C9182FF15C0B8E0BB16F9
:1076900091F0E6E0BE1611F087E901C085E9D80156
:1076A0008C9380E211968C938EEF8B0D8093392A08
:1076B00060E170E049C081E080933A2A8B2D90E030
:1076C0000697982F990F890F8C5F8093382AF801BD
:1076D000808180932D2A3EC06115710531F481E0CF
:1076E0008093392A0E947F2833C0C80139D97C0190
:1076F000BC01C80162D981110FC0C701089667E0BB
:1077000070E00E942045462FE091552BF091562BBA
:10771000B80181EC199508C0B701C801D3D863E05E
:10772000C801B5D9892BD9F282ECD8018C9361E0DC
:10773000C801ADD9F801818392838AE08093392A08
:1077400010923A2A68E170E0C8014ED87C0102C06C
:10775000E12CF12C80913A2A882309F400C280910F
:10776000392A9AEF980F933008F04CC0D801FC905A
:10777000F5FAFF24F0F8E1EEAE2EEFE0BE2EE12C9C
:1077800047E650E0B501CE0101960E94A8458B81E5
:10779000882349F029813A8180912B2A90912C2AC3
:1077A00028173907B9F48D81882329F09C818091AD
:1077B0002D2A98130FC08F89882311F0FF2051F0D4
:1077C000E0911B2A81E08E0F80931B2AF0E0E45E9B
:1077D000F54DE082E394B7E6AB0EB11CEFE0EE129C
:1077E000CFCFFF2009F493C080EED8018C9380E8BE
:1077F00011968C9362E0C8014AD9F8018283938381
:1078000089E0A6C0893009F082C0B601C801A8D8B5
:107810007C01BC01C801D1D881110FC0C7010896F5
:1078200067E070E00E942045462FE091552BF091D3
:10783000562BB80181EC1995BEC0B701C80142D8DA
:107840006C01D8016C91262F30E073E096958795F6
:107850007A95E1F702972817390729F46E5FC80176
:1078600016D9892B69F082ECF801808361E0C801A8
:107870000ED9D80111968C93119712969C93A4C09F
:10788000F12C67E6E62E5801FFEFAF1ABF0A809190
:107890001B2AF816E0F5EF2DF0E0E45EF54D60816F
:1078A000E69EB00111246F51704F47E650E0CE01C3
:1078B00001960E94A8458F89882339F14E8950E0AE
:1078C000F801808190E001974817590739F4B50114
:1078D000CE0106960E94C945892BB9F020911B2A3A
:1078E000422F50E0415051093F2D832F90E08417E3
:1078F00095073CF4FC01E45EF54D818180833F5F98
:10790000F4CF215020931B2AFA94F394C0CF809196
:10791000392A9AEF980F9430F0F490911B2A2CE1B9
:107920003AE2F9018E2F821B891708F069C0819114
:1079300084508230B8F782E0D8018C9380E61196AB
:107940008C9362E0C801A3D8F801828393838BE013
:107950008093392AB0CD8B3009F052C0C114D104C4
:1079600009F44CC0B601C8010E94B0347C01BC01CE
:10797000C80123D881110FC0C701089667E070E0E5
:107980000E942045462FE091552BF091562BB801CF
:1079900081EC19950EC0B701C8010E94623453E012
:1079A000969587955A95E1F7682FC80170D8892B6D
:1079B00099F010921B2A82ECD8018C9361E0C801E7
:1079C00066D8F801818392838AE08093392A1092E5
:1079D0003A2A68E170E071CDD80113968C91882322
:1079E00031F0813059F480931B2A85E004C081E096
:1079F00080931B2A84E080931C2A02C010921B2AC9
:107A000080911B2A811103C06CEE70E213C081309B
:107A1000A9F460911C2AB7E66B9FB0011124685F3E
:107A20007F4E40E450E0CE0101960E94A845BE0181
:107A30006F5F7F4F85E60E94B22068C0912C80E086
:107A400090E000E010E027E6822E7E013FEFE31A8F
:107A50003DEFF30A3FEFC32E30E2D32EA12C42E0DC
:107A6000B42E20911B2A921680F50130E2E01E0709
:107A700020F0081B190BF12C2EC0E92DF0E0E45E7C
:107A8000F54D6081869EB0011124685F7F4E40E411
:107A900050E0C7010E94A845FF92EF92DF92CF927B
:107AA000C501801B910B9F938F9381E090E08C0F19
:107AB0009D1F800F911F9F938F930E940946080F6F
:107AC000191F9394CDBFDEBFCCCF0130A2E01A07BF
:107AD00080F6FF24F394EDEFFFEFEC0FFD1FE00FB6
:107AE000F11F8EE28083EEEFFFEFEC0FFD1FE00F42
:107AF000F11F1082BE016F5F7F4F85E60E94B220AA
:107B0000F11004C086E091E20E945C1788E691E2E1
:107B10000E945C1762E070E08BE29AE20E94D02043
:107B20008FE691E20E945C176091382A70E08EE245
:107B30009AE20E94D02085E791E20E945C1761E002
:107B400070E08DE29AE20E94D0201092D929109222
:107B50001B2A0E94482110923A2AE12CF12CC701DD
:107B6000CF5BDD4FCDBFDEBFDF91CF911F910F9176
:107B7000FF90EF90DF90CF90BF90AF909F908F904D
:107B80000895FF920F931F93CF93DF93CDB7DEB786
:107B9000EA97CDBFDEBF0FEA1EE288E0F82EF00EB6
:107BA00091D2F80181938F01FE12FACF0E94101832
:107BB00004D3882309F4F7C08091AF2E9091B02EA2
:107BC000953009F46FC030F4913069F168F093306A
:107BD00051F1E9C0983009F4C2C0993009F4C8C025
:107BE000963009F0E0C072C0803891F0823809F018
:107BF000DAC08091B32E8F7085D2E091B92EF091CA
:107C0000BA2E118112FB112710F980E07BD206C039
:107C10001091AB2E8091AC2E81111260E8D2812F91
:107C200061D280E0A1C0282F2D7F09F0BCC088233D
:107C300019F0823061F0B7C08091B12E813009F027
:107C4000B2C0933009F080E08093AC2E27C08091C1
:107C5000B12E811123C0E091B32E1E2F1F7009F4A5
:107C6000A2C0812F4FD28091B02E833011F4EBD27D
:107C700015C0E091B92EF091BA2E81818B7F81835E
:107C800024E8129FF0011124E350F14D1082E0919D
:107C9000B92EF091BA2E80818E7F808380E032D21F
:107CA000A6D264C081117FC01091B12E1F779FD2E0
:107CB000A1D35DD28823E9F31093C304111102C04C
:107CC00082E001C083E08093AE2E6DC08058823088
:107CD00008F069C08091B12E9091B22E8C3DE3E006
:107CE0009E0761F583E08A838AE389834FB7F8941E
:107CF000DE01139620E038E052E05093CA01E32FF2
:107D0000F0E0E4911092CA0120FF03C0E295EF7009
:107D10003F5FEF708E2F90E0EA3010F0C79601C001
:107D2000C0968D939D932F5F2C3139F74FBF5FD253
:107D30006AE370E0CE010196A3D00FC0AE014F5FA1
:107D40005F4F6091B32E0E94120C8C01892B59F168
:107D50004ED2B80189819A810FD1A5D124C0803833
:107D600011F545D28091AA2EBDD184D143D31BC039
:107D7000811119C08091B12E8230A8F438D280913F
:107D8000B12E8093AA2E36D38091AA2E811106C0DF
:107D90008091C304811102C081E001C084E080931E
:107DA000AE2E0E940C1809D2882311F020D24BD29B
:107DB000EA96CDBFDEBFDF91CF911F910F91FF906B
:107DC00008950895CF938091AE2E882351F0C091ED
:107DD000BB2E80E097D1F1D18111D3DE8C2FCF91D2
:107DE00091C1CF910895CF92DF92EF92FF920F93BE
:107DF0001F93CF93DF93EC018B017A0111D3811193
:107E000036C0E114F10439F0F70180819181081B3B
:107E1000190BC80FD91FC12CD12C0115110531F137
:107E20008091B72E9091B82EFC01EF5BFF4F20811F
:107E300031978081281790F01DD1C4DFE114F1043F
:107E400049F0F70180819181C80ED91EC082D1828C
:107E500085E00DC0E5D2882301F309C0899142D1A4
:107E600001501109FFEFCF1ADF0AD7CF80E0DF9171
:107E7000CF911F910F91FF90EF90DF90CF900895D9
:107E8000DF92EF92FF920F931F93CF93DF93D82F40
:107E9000C92F8B018091BB2E806834D12091B52EE3
:107EA0003091B62E2017310728F00115110519F46D
:107EB000E1D001C08901ED2EFC2ED12C0115110558
:107EC00009F440C08091AE2E811102C082E04CC006
:107ED000853011F483E048C070D1882311F081E02F
:107EE00043C051D181113CC042D1882339F3209144
:107EF000BB2E8091B72E9091B82EFC0127FF05C0B4
:107F0000EF5BFF4FC081D0E013C0E05CFF4FC0814A
:107F100031968081D0E0C81BD1090AC0C830D10594
:107F200050F4F70181917F01DDD0015011092196B4
:107F30000115110599F7DD24D394289709F0D12C68
:107F400099D0BCCFD110BECF0BC08091AE2E88236C
:107F500009F4BCCF853009F4BDCF2FD18111BFCF3B
:107F600012D1882391F380E0DF91CF911F910F917F
:107F7000FF90EF90DF900895DF92EF92FF920F93C2
:107F80001F93CF93DF93D82FC92F8B018091BB2EE6
:107F90008068B8D02091B52E3091B62E20173107C9
:107FA00028F00115110519F465D001C08901ED2EE5
:107FB000FC2ED12C0115110509F442C08091AE2E82
:107FC000811102C082E04EC0853011F483E04AC0C6
:107FD000F4D0882311F081E045C0D5D081113EC096
:107FE000C6D0882339F32091BB2E8091B72E909173
:107FF000B82EFC0127FF05C0EF5BFF4FC081D0E02A
:1080000015C0E05CFF4FC08131968081D0E0C81B75
:10801000D1090CC0C830D10560F4F701849162D059
:10802000FFEFEF1AFF0A0150110921960115110502
:1080300089F7DD24D394289709F0D12C1BD0BACF2F
:10804000D110BCCF0BC08091AE2E882309F4BACFDB
:10805000853009F4BBCFB1D08111BDCF94D0882336
:1080600091F380E0DF91CF911F910F91FF90EF90FE
:10807000DF900895E091B92EF091BA2EA091B72E1D
:10808000B091B82EAF5BBF4F8C9190E08283938309
:1080900080818D798083E091B72EF091B82EEF5BCF
:1080A000FF4F10820895E091B92EF091BA2E808191
:1080B0008D798083E091B72EF091B82EEF5BFF4F62
:1080C000108208958091B72E9091B82EFC01EF5B3D
:1080D000FF4F208131E0320F3083FC01E20FF11DB0
:1080E000808108952091B72E3091B82EF901EF5B71
:1080F000FF4F908141E0490F4083F901E90FF11DE5
:10810000808308958093BB2E482F4F7050E060917C
:10811000C6047091C7049A0194E0220F331F9A9508
:10812000E1F7E4E887FF11C0E49FC001E59F900DEF
:1081300011248250914D8093B72E9093B82EC9018F
:1081400008969B01280F391F0DC0E49FC001E59FD1
:10815000900D11248454914D8093B72E9093B82E96
:10816000260F371F2093B92E3093BA2E0895809191
:10817000BB2E8068C7DFE091B92EF091BA2E8081C6
:108180008695817008958091BB2E8F77BBDFA0917B
:10819000B92EB091BA2E8C9185FF0DC0E091B72E0B
:1081A000F091B82E12968D919C911397E05CFF4F41
:1081B000808381E0089580E008958091BB2E8F77C1
:1081C000A1DFA091B92EB091BA2E8C9184FF0DC081
:1081D000E091B72EF091B82E12968D919C91139745
:1081E000E05CFF4F808381E0089580E008958091F6
:1081F000BB2E8F7787DFE091B92EF091BA2E808168
:108200008D788083E091B92EF091BA2E80818160C3
:108210008083E091B72EF091B82EEF5BFF4F108274
:108220008091BB2E80686EDFE091B92EF091BA2E5E
:10823000808181608083E091B72EF091B82EEF5B52
:10824000FF4F10820895E091B92EF091BA2E8181EE
:1082500084608183E091B92EF091BA2E8181807C77
:10826000803459F48091BB2E80584CDFE091B92EB8
:10827000F091BA2E81818460818308951F93CF93FA
:10828000DF931F921F92CDB7DEB7182F4A83698301
:1082900039DFE091B92EF091BA2E1182E091B92E1A
:1082A000F091BA2E812F881F8827881F880F80831E
:1082B000E091B92EF091BA2E69816183E091B92ED7
:1082C000F091BA2E128213822091B72E3091B82EDF
:1082D00024833583110F110B4A814123F901E05C9E
:1082E000FF4F40833196108281E00F900F90DF9115
:1082F000CF911F910895AF92BF92CF92DF92EF92EC
:10830000FF920F931F93CF93DF93A62E8C017C01D6
:1083100084E0E80EF11CB12CBA1409F443C0F80152
:10832000D081DD23C1F1C180D280F70131978081F6
:10833000F7019081923010F498E001C098E128E0B4
:1083400030E0C0E02C153D0520F4CF5F220F331F35
:10835000F9CFC92B9D2F9F70963010F080E023C07D
:10836000CF7EF1E4CF16D104C8F7882321F0813005
:1083700021F4C06C0AC0C06403C0C068811105C08C
:108380004C2D6C2F80E88D0F79DF4C2D6C2F8D2FAD
:1083900075DF882319F3B3940B5F1F4F85E0E80E58
:1083A000F11CBACF81E0DF91CF911F910F91FF9027
:1083B000EF90DF90CF90BF90AF90089580E090E075
:1083C000E091C604F091C7049C0144E0220F331FE2
:1083D0004A95E1F7E20FF31F11864091C6045091D0
:1083E000C704FA01E20FF31F11820196863091054E
:1083F00039F708958091AF2E87FF0DC0C4DE81113B
:1084000005C08091AE2E8111F9CF09C04CCE80916C
:10841000AE2E882321F0ABDE8823C9F32BCE08953E
:108420000F931F93CF93E091C604F091C704E05AD5
:10843000FF4F00811181C4E68091BB2E87FF0AC0E7
:1084400096DE811105C08091AE2E811105C021C03C
:1084500080E024C098DEF5CF8530E9F0E091B92EB8
:10846000F091BA2E818182FD18C0E091C604F0918E
:10847000C704E05AFF4F8081918180179107E1F294
:108480002FEF2C0FCC2319F08C01C22FD5CF84E015
:1084900005C082E003C083E001C081E0CF911F915D
:1084A0000F91089563D069D0E0ECF4E081818E7F74
:1084B000818380818F7780831092AD2E0895CF9332
:1084C000DF93E0E4F0E014828481836084834ED003
:1084D00054D0C0ECD4E088818F778883888180680D
:1084E00088831092AE2E1092AA2E1092AC2E10926B
:1084F000AB2E88818064888348E068E480E8BEDE33
:1085000048E068E480E0BADE8885806488878981F5
:1085100081608983DF91CF910895CF93DF933FB737
:10852000F894C0ECD1E022E02A87EAE1F0E0E4919F
:10853000A0ECB4E0DA96EC93DA97EBE1F0E0E491AA
:10854000DB96EC93DB971A8685ED91E38E7F16968A
:108550008D939C93179785E18C9318962C933FBF2E
:1085600081E08093AD2EDF91CF91A9CFE0ECF4E0D4
:1085700080858370808711860895E0ECF4E08FEFAA
:108580008287848708951F920F920FB60F9211244D
:1085900008B60F9218BE09B60F9219BE0BB60F920D
:1085A0001BBE2F933F934F935F936F937F938F9354
:1085B0009F93AF93BF93EF93FF938091CA0487FF7C
:1085C00008C08091C80487FF04C080E88093CA0473
:1085D000F8DB8091CA0486FF07C080E48093CA0458
:1085E0001092AE2E0E94FB178091CA0485FF14C022
:1085F00080E28093CA048091AA2E882311F084E03F
:1086000007C08091C304811102C081E001C083E0F2
:108610008093AE2E0E94EA178091CA0484FF14C092
:1086200080E18093CA0482E08093AE2E1092AA2E3D
:108630001092C304C3DE48E068E480E81FDE48E02F
:1086400068E480E01BDEBDDBFF91EF91BF91AF914D
:108650009F918F917F916F915F914F913F912F915A
:108660000F900BBE0F9009BE0F9008BE0F900FBE6B
:108670000F901F901895CF93DF93EC01FC0170963B
:108680008BE0DF011D928A95E9F782E08C83898770
:1086900083E08E8761E0CE0101962DDE882361F0B4
:1086A00061E0CE01069627DE882331F061E0CE013D
:1086B0000B96DF91CF911FCE80E0DF91CF9108958F
:1086C0000F931F93CF93DF932091AE2E2430E1F4CC
:1086D000FC010489158926893789012B022B032B7C
:1086E00099F0EB0181810EDDFE0101900020E9F798
:1086F0003197BF016C1B7D0B40E050E0CE01DF9154
:10870000CF911F910F916FCB82E0DF91CF911F919D
:108710000F9108950F931F93CF93DF93FC018091E6
:10872000AE2E8430A9F484899589A689B789892BCE
:108730008A2B8B2B69F08A01EB018181E3DC40E01D
:1087400050E0B801CE01DF91CF911F910F914BCB3B
:1087500082E0DF91CF911F910F910895CF93FC019B
:108760008091AE2E843001F584899589A689B789D8
:10877000892B8A2B8B2BC1F0C62F8181C3DC2091E2
:10878000B72E3091B82EF901EF5BFF4F90813197F2
:108790008081981720F48C2FA5DC80E006C06ADC6D
:1087A0003FDE8823C1F301C082E0CF910895CF93CB
:1087B000DF932091AE2E243091F5FC014489558938
:1087C00066897789452B462B472B49F181819ADCB5
:1087D0008091BB2E2091B72E3091B82EF90187FFE2
:1087E00005C0EF5BFF4F808190E008C0E05CFF4F69
:1087F00080813196408190E0841B9109892B69F03A
:10880000F901EF5BFF4FD0813197C08133DCDC177A
:1088100020F006DE811104C02DDC80E001C082E082
:10882000DF91CF910895CF93DF932091AE2E243026
:1088300099F4FC014489558966897789452B462B33
:10884000472B51F0EC0181815DDC91DC882321F024
:10885000CE01DF91CF91ABCFDF91CF910895CF9330
:10886000DF932091AE2E243019F08FEF9FEF46C09A
:10887000FC014489558966897789452B462B472B0E
:10888000A1F386813FDC7FDC882379F38091BB2EC6
:108890002091B72E3091B82EF90187FF05C0EF5B0C
:1088A000FF4F808190E008C0E05CFF4F80813196EF
:1088B000208190E0821B9109892B21F003DCC82FD5
:1088C000D0E002C0CFEFDFEF2091BB2E8091B72E1A
:1088D0009091B82EFC0127FF05C0EF5BFF4F208170
:1088E00030E008C0E05CFF4F20813196808130E0AD
:1088F000281B3109232B09F4D6DBCE01DF91CF9160
:1089000008950895FF920F931F93CF93DF93EC0187
:1089100054DC882309F48EC0888190E02091B32E26
:108920003091B42E2817390709F084C08091B02EF9
:10893000813259F018F4803249F17CC0823209F456
:1089400057C0833209F467C075C08091AF2E813A59
:1089500009F070C04CDC0BDC8823E9F38C89FD88BE
:108960000E891F89BFDB8F2DBDDB802FBBDB812FE5
:10897000B9DB888DB7DB898DB5DB8A8DB3DB7ADB1C
:10898000DF91CF911F910F91FF9034CD8091AF2E49
:10899000813209F04FC02BDCF6DB811105C08091DC
:1089A000AE2E8111F9CF46C08DDB082F8BDB182F3F
:1089B00089DBF82E87DB4F2D50E060E070E0BA01D4
:1089C00055274427782B402B512B4C8B5D8B6E8B7E
:1089D0007F8B78DB888F76DB898F74DB8A8F63DB14
:1089E00009DDCE01DF91CF911F910F91FF9089CFCB
:1089F0008091AF2E8132F1F4FADBFCDC8091B12E54
:108A00009091B22E888B998BCE01DF91CF911F91DF
:108A10000F91FF9076CF8091AF2E813259F4E7DB32
:108A2000E9DC6091B12ECE01DF91CF911F910F91C2
:108A3000FF9067CFDF91CF911F910F91FF90089525
:108A4000AA1BBB1B51E107C0AA1FBB1FA617B70774
:108A500010F0A61BB70B881F991F5A95A9F7809590
:108A60009095BC01CD010895B7FF04C003D0821BCF
:108A7000930B089509D0A59F900DB49F900DA49FCE
:108A8000800D911D11240895A29FB001B39FC001D4
:108A9000A39F700D811D1124911DB29F700D811D2A
:108AA0001124911D08958F929F92AF92BF92CF9201
:108AB000DF92EF92FF92CF93DF93EC01688179818F
:108AC0008A819B81611571058105910521F464E21C
:108AD00079ED8BE597E02DE133EF41E050E0E2D610
:108AE00049015A019B01AC01A7EAB1E4C3DF6B0164
:108AF0007C01ACEEB4EFA5019401B8DFDC01CB0141
:108B00008C0D9D1DAE1DBF1DB7FF03C00197A109B0
:108B1000B04888839983AA83BB839F77DF91CF91E5
:108B2000FF90EF90DF90CF90BF90AF909F908F908D
:108B30000895B9CF80E290E2B6CFA0E0B0E0809394
:108B4000202090932120A0932220B09323200895E9
:108B5000FB01DC0102C005900D9241505040D8F756
:108B60000895FB01DC018D91059080190110D9F366
:108B7000990B0895FB01DC014150504048F00590ED
:108B80000D920020C9F701C01D9241505040E0F7FE
:108B90000895FB01DC0104C08D910190801921F43E
:108BA00041505040C8F7881B990B0895FB01DC0128
:108BB00002C001900D9241505040D8F708956817B7
:108BC000790768F4FB01DC01E40FF51FA40FB51F62
:108BD00002C002900E9241505040D8F70895E6CF5F
:108BE000DC0101C06D9341505040E0F70895FC0155
:108BF0008191861721F08823D9F799270895319715
:108C0000CF010895FB01DC0101900D920020E1F7F6
:108C100008950F931F93CF93DF93CDB7DEB72E97B1
:108C2000CDBFDEBF0E891F89888D998D26E02C83EC
:108C300009831A8397FF02C080E090E801978D8333
:108C40009E83AE01445E5F4F6A8D7B8DCE0101969F
:108C500067D04D815E8157FD0AC02F81388542174C
:108C600053070CF49A01F801E20FF31F10822E96BD
:108C7000CDBFDEBFDF91CF911F910F9108950F936C
:108C80001F93CF93DF93CDB7DEB72E97CDBFDEBF57
:108C90000E891F89888D998D2EE02C8309831A8374
:108CA00097FF02C080E090E801978D839E83AE011C
:108CB000445E5F4F6A8D7B8DCE01019631D04D8130
:108CC0005E8157FD0AC02F813885421753070CF487
:108CD0009A01F801E20FF31F10822E96CDBFDEBF7E
:108CE000DF91CF911F910F910895CF93DF93CDB76F
:108CF000DEB72E97CDBFDEBF85E08C838C899D8942
:108D000089839A83AE01485E5F4F6E897F89CE0169
:108D100001968FD32E96CDBFDEBFDF91CF91089500
:108D20002F923F924F925F926F927F928F929F927B
:108D3000AF92BF92CF92DF92EF92FF920F931F9369
:108D4000CF93DF93CDB7DEB72C97CDBFDEBF7C01CD
:108D50006B018A01FC0116821782838181FFB0C1F9
:108D6000CE0101964C01F7019381F60193FD8591A7
:108D700093FF81916F01882309F49EC1853239F4F4
:108D800093FD859193FF81916F01853221F4B701A5
:108D900090E0D6D4E8CF512C312C20E02032A0F442
:108DA0008B3269F030F4803259F0833269F42061FB
:108DB0002CC08D3239F0803339F4216026C0226016
:108DC000246023C0286021C027FD27C030ED380F64
:108DD0003A3078F426FF06C0FAE05F9E300D112489
:108DE000532E13C08AE0389E300D1124332E20629A
:108DF0000CC08E3221F426FD5FC1206406C08C3683
:108E000011F4206802C0883641F4F60193FD859183
:108E100093FF81916F018111C1CF982F9F7D955450
:108E2000933028F40C5F1F4FFFE3F9830DC08336A6
:108E300031F0833771F0833509F057C021C0F80154
:108E4000808189830E5F1F4F44244394512C540129
:108E500014C03801F2E06F0E711CF801A080B180DF
:108E600026FF03C0652D70E002C06FEF7FEFC501E4
:108E70002C871DD42C0183012C852F77222E16C020
:108E80003801F2E06F0E711CF801A080B18026FF5E
:108E900003C0652D70E002C06FEF7FEFC5012C8726
:108EA000FBD32C012C852068222E830123FC19C0C2
:108EB000832D90E048165906A0F4B70180E290E0B7
:108EC0003FD43A94F5CFF50127FC859127FE819197
:108ED0005F01B70190E034D431103A94F1E04F1AB9
:108EE00051084114510479F7DEC0843611F08936F7
:108EF00031F5F80127FF07C060817181828193817C
:108F00000C5F1F4F08C060817181072E000C880B19
:108F1000990B0E5F1F4F2F76722E97FF09C0909509
:108F20008095709561957F4F8F4F9F4F2068722E6F
:108F30002AE030E0A40155D4A82EA81843C08537F4
:108F400029F42F7EB22E2AE030E025C0F22FF97FDF
:108F5000BF2E8F36C1F018F4883579F0ADC0803758
:108F600019F0883721F0A8C02F2F2061B22EB4FE4F
:108F70000DC08B2D8460B82E09C024FF0AC09F2F1E
:108F80009660B92E06C028E030E005C020E130E050
:108F900002C020E132E0F801B7FE07C060817181B4
:108FA000828193810C5F1F4F06C06081718180E0D8
:108FB00090E00E5F1F4FA40114D4A82EA818FB2D1B
:108FC000FF777F2E76FE0BC0372D3E7FA51450F421
:108FD00074FE0AC072FC08C0372D3E7E05C0BA2C54
:108FE000372D03C0BA2C01C0B52C34FF0DC0FE01D3
:108FF000EA0DF11D8081803311F4397E09C032FF02
:1090000006C0B394B39404C0832F867809F0B39458
:1090100033FD12C030FF06C05A2CB31418F4530CA1
:109020005B18B32CB31460F4B70180E290E03C8786
:1090300087D3B3943C85F6CFB31410F43B1801C02A
:10904000312C34FF11C0B70180E390E03C8778D326
:109050003C8532FF16C031FD03C088E790E002C0B6
:1090600088E590E0B7010CC0832F867851F031FF7E
:1090700002C08BE201C080E237FD8DE2B70190E0D3
:109080005FD3A51430F4B70180E390E059D35A942C
:10909000F8CFAA94F401EA0DF11D8081B70190E0A8
:1090A0004FD3A110F6CF332009F45DCEB70180E293
:1090B00090E046D33A94F7CFF7018681978102C0BA
:1090C0008FEF9FEF2C96CDBFDEBFDF91CF911F9129
:1090D0000F91FF90EF90DF90CF90BF90AF909F9057
:1090E0008F907F906F905F904F903F902F9008955A
:1090F00020FD09C0FC0123FD05C022FF02C07383CF
:10910000628351834083089544FD10C046FD10C022
:10911000DB01FC01AA0FBB1FEE1FFF1F1094D1F74C
:109120006A0F7B1F8E1F9F1F31E003C033E001C019
:1091300034E0660F771F881F991F3150D1F7620FF7
:10914000711D811D911D08950F931F93CF93DF9380
:109150008C01C801B7D2EC0197FD06C08AD2892BD9
:10916000C1F7B801CE0124D3CE01DF91CF911F9179
:109170000F9108958F929F92AF92BF92CF92DF92FC
:10918000EF92FF920F931F93CF93DF931F92CDB770
:10919000DEB78C01C62E7A01298394D2AC01552703
:1091A00029814B32510521F04D32510561F420687F
:1091B000CA94C11002C080E06FC0C801298382D266
:1091C000298197FDF8CF322F3D7FD32E322F307378
:1091D00039F5803329F5BB24BA94BC0C09F449C095
:1091E000C80129836FD2298197FD43C0382F3F7D65
:1091F000383561F48D2D8264D82ECA94CA94CC205F
:10920000C1F1C8015FD297FF0BC033C026FF04C075
:109210002D2D2260D22E03C03D2D3261D32ECB2CBA
:10922000812C912C540120ED280F283078F0D4FEA9
:1092300003C0B801BDD21AC02A3040F0D6FEF9CF23
:109240002F7D3FEE320F3630A0F727504D2DC50150
:10925000B4015ADF4B015C018D2D8260D82ECA9477
:10926000CC2051F0C8012ED297FFDDCFD1FC04C035
:10927000A2CF812C912C5401D7FE08C0B094A094A9
:1092800090948094811C911CA11CB11C2D2DB501C2
:10929000A401C7012DDF81E00F90DF91CF911F91D5
:1092A0000F91FF90EF90DF90CF90BF90AF909F9085
:1092B0008F9008956F927F928F929F92AF92BF92FC
:1092C000CF92DF92EF92FF920F931F93CF93DF9392
:1092D000CDB7DEB7A197CDBFDEBF5C017A01CE016D
:1092E00001966C0180E2F60111928A95E9F7F50189
:1092F000838040E050E0912C712C70E0A1E0B0E060
:10930000F90183FC859183FE81918F01982F9F0144
:10931000811103C080E090E07AC08E3519F44115C8
:10932000510549F1E72FF0E0E417F5073CF48D35DE
:1093300059F18D3219F4772001F103C0711001C089
:10934000982E892F8695869586958601080F111D82
:10935000892F87703D0101C0660C8A95EAF7F801F4
:10936000808186298083991559F0991510F49F5FA3
:10937000E8CF9150E6CF71E004C07724739401C028
:10938000712C4F5F5F4FBCCF772019F08E818062C8
:109390008E83711103C09924939416C0F6019E0127
:1093A0002F5D3F4F808180958193E217F307D1F7BE
:1093B000F2CFE114F10429F0F7018083C70101968F
:1093C0007C016150912CE9F0C50169A37BD169A1B1
:1093D00097FD15C0282F269526952695F601E20FB4
:1093E000F11D208130E0AC014770552702C0359552
:1093F00027954A95E2F720FDDCCFB501D9D1911030
:1094000089CFE114F10411F0F7011082C801A1968F
:10941000CDBFDEBFDF91CF911F910F91FF90EF90F5
:10942000DF90CF90BF90AF909F908F907F906F9084
:1094300008954F925F927F928F929F92AF92BF92C8
:10944000CF92DF92EF92FF920F931F93CF93DF9310
:109450001F92CDB7DEB76C012B015A01FC011682B9
:109460001782712CF601F380F201F3FC8591F3FE73
:109470008191382F2F01882309F4E5C090E03983CA
:10948000F8D03981892B19F0C6015EDEEBCF353279
:1094900041F4F201F3FC3591F3FE31912F013532A5
:1094A00059F4C60139830ED1398197FDCAC03817E6
:1094B000C9F2B6017DD1C7C03A3239F4F3FC359117
:1094C000F3FE31912F0151E001C050E0420110E064
:1094D00020ED230F2A3088F45260612F70E080E085
:1094E00090E040E2598310DE162FF401F3FC359131
:1094F000F3FE31914F015981EBCF052F232F24012A
:1095000051FF03C0111102C09EC01FEF383619F081
:109510003C3659F011C0F401F3FC2591F3FE219182
:109520002F01283649F4052F08600460F201F3FC8E
:109530002591F3FE21912F01222309F484C0622F8B
:1095400070E08AEE95E129839CD02981892B09F46A
:109550007AC000FD07C0F501E080F180C5010296E8
:109560005C0102C0E12CF12C2E3649F4F601468153
:10957000578160E070E0202FC701BADD73CF23363A
:1095800089F401FF11E0C6019DD097FD5AC0E11496
:10959000F10429F0F7018083C70101967C01115085
:1095A00091F74BC02B3551F49201A701612FC601F1
:1095B00081DE2C01892B09F040C03AC0C601298305
:1095C000C3DD298197FD3DC02F3641F128F42436B3
:1095D00019F1293631F124C0233769F02537E1F03C
:1095E0001FC0E114F10429F0F7018082C701019640
:1095F0007C01115059F0C60165D04C0197FD06C0A1
:1096000038D0892B71F3B601C401D2D0E114F10432
:10961000A1F0F701108211C0006203C0006101C017
:109620000064202FA701612FC601A4DD811105C0B0
:10963000F6018381807329F406C000FD13CF739473
:1096400011CF772019F0872D90E002C08FEF9FEFA8
:109650000F90DF91CF911F910F91FF90EF90DF90CE
:10966000CF90BF90AF909F908F907F905F904F90E2
:109670000895911114C1803219F089508550D0F7A6
:109680000895FC010590061621F00020D9F7C001CD
:1096900008953197CF010895FC0105906150704005
:1096A0000110D8F7809590958E0F9F1F0895FC01AB
:1096B0006150704001900110D8F7809590958E0F01
:1096C0009F1F0895CF93DF93EC012B8120FF33C0C0
:1096D00026FF0AC02F7B2B838E819F8101968E836C
:1096E0009F838A8190E029C022FF0FC0E881F98121
:1096F0008081082E000C990B009719F420622B83AF
:109700001AC03196E883F9830EC0EA85FB85199566
:1097100097FF09C02B81019611F080E201C080E122
:10972000822B8B8308C02E813F812F5F3F4F2E837A
:109730003F83992702C08FEF9FEFDF91CF9108956C
:109740000F931F93CF93DF93FB01238121FD03C070
:109750008FEF9FEF28C022FF16C0468157812481DA
:1097600035814217530744F4A081B1819D012F5FD9
:109770003F4F208331838C93268137812F5F3F4F6A
:109780002683378310C0EB01092F182F0084F18541
:10979000E02D1995892BE1F68E819F8101968E83AC
:1097A0009F83812F902FDF91CF911F910F9108956B
:1097B000FB01238120FF12C026FD10C08F3F3FEF29
:1097C000930761F082832F7D206423832681378174
:1097D0002150310926833783992708958FEF9FEF12
:1097E0000895FA01AA27283051F1203181F1E89437
:1097F0006F936E7F6E5F7F4F8F4F9F4FAF4FB1E084
:109800003ED0B4E03CD0670F781F891F9A1FA11D7E
:10981000680F791F8A1F911DA11D6A0F711D811D7F
:10982000911DA11D20D009F468943F912AE0269F44
:1098300011243019305D3193DEF6CF010895462FA3
:109840004770405D4193B3E00FD0C9F7F6CF462F84
:109850004F70405D4A3318F0495D31FD40524193ED
:1098600002D0A9F7EACFB4E0A695979587957795AA
:109870006795BA95C9F700976105710508959B0131
:10988000AC010A2E06945795479537952795BA95BA
:10989000C9F7620F731F841F951FA01D0895992794
:1098A00088270895052E97FB16F400940FD057FDD6
:1098B00005D014D007FC02D046F408C0509540955E
:1098C000309521953F4F4F4F5F4F0895909580956C
:1098D000709561957F4F8F4F9F4F0895A1E21A2E8B
:1098E000AA1BBB1BFD010DC0AA1FBB1FEE1FFF1F44
:1098F000A217B307E407F50720F0A21BB30BE40B94
:10990000F50B661F771F881F991F1A9469F76095DA
:109910007095809590959B01AC01BD01CF01089594
:04992000F894FFCFE9
:1099240000400F00831000000104100000018208B1
:109934000000010000000000000000000000900191
:10994400010000000000000093229A229A22A6221D
:10995400B222BC22D922E7221023132317239225F3
:10996400F42409250D252225532566259325000178
:1099740000010000000000000001000101010101DC
:1099840001000100010000000101000101010001CA
:1099940001010000000100000100010100010000BC
:1099A40000020200000200020202020000020000A3
:1099B400000404000004000404040400000400087B
:1099C400080800000008000008000808000800005B
:1099D40000101000001000101010100000102535A9
:1099E4006400546F6F206D616E7920646174612E20
:1099F400000D0A504152495459204552524F5200C9
:109A04000D0A504152495459204F4B00556E6B6E0C
:109A14006F776E206361726420747970652E0025FF
:109A240073206F7220005468657265206973206129
:109A340074206C65617374206F6E65206D6F726540
:109A4400206361726420747970652063616E646957
:109A5400646174652C206275742074686572652075
:109A6400776173206E6F7420656E6F7567682074FC
:109A740065726D696E616C206275666665722073CD
:109A8400706163652E0D0A00415451413A09005535
:109A940049443A090053414B3A09004E4F2044418E
:049AA4005441000029
:020000021000EC
:1000000000000000000000000000000000000000F0
:1000100000000000000000000000000000000000E0
:1000200000000000000000000000000000000000D0
:1000300000000000000000000000000000000000C0
:00000001FF
